:020000040002F8
:10600000405C0020C1630200C9630200CB63020050
:10601000CD630200CF630200D163020000000000E4
:10602000000000000000000000000000D363020038
:10603000D563020000000000D7630200D9630200AC
:10604000AD670200DB6302000D6A0200DB63020041
:10605000DB630200DB63020095650200DB63020084
:10606000DB630200DB630200DB630200DB63020030
:10607000DB630200DB630200DB630200DB63020020
:10608000DB63020005680200DB630200DB630200E1
:1060900029680200DB6302002D680200DB63020056
:1060A000DB630200DB630200DB630200DB630200F0
:1060B000DB630200DB630200000000000000000060
:1060C000DB630200DB630200DB630200DB630200D0
:1060D000DB630200DB630200DB630200DB630200C0
:1060E000DB630200DB630200DB63020000000000F0
:1060F00000000000DB63020000000000DB63020020
:10610000000000000000000000000000000000008F
:10611000000000000000000000000000000000007F
:10612000000000000000000000000000000000006F
:10613000000000000000000000000000000000005F
:10614000000000000000000000000000000000004F
:10615000000000000000000000000000000000003F
:10616000000000000000000000000000000000002F
:10617000000000000000000000000000000000001F
:10618000000000000000000000000000000000000F
:1061900000000000000000000000000000000000FF
:1061A00000000000000000000000000000000000EF
:1061B00000000000000000000000000000000000DF
:1061C00000000000000000000000000000000000CF
:1061D00000000000000000000000000000000000BF
:1061E00000000000000000000000000000000000AF
:1061F000000000000000000000000000000000009F
:10620000DFF80CD000F088F90048004791A70200A1
:10621000405C002030B450E8012F93B2C48923447D
:106220008489A34228BF1B1B0489A34202BFBFF37A
:106230002F8F002007E0C3EA020340E80134002C5E
:10624000E9D14FF001000A6030BC704750E8012FDF
:10625000C2EA024240E801210029F7D1704730B478
:1062600050E8022F1FFAA2F3C488A34202BFBFF373
:106270002F8F00200DE0C48923448489A34228BFC6
:106280001B1BC2EA034340E80234002CE8D14FF064
:1062900001000A6030BC704750E8022FC2EA224277
:1062A00040E802210029F7D17047034653E8022F46
:1062B000D988B2EB324F4FF0000017BF92B241EADB
:1062C000014142EA014104E05A68B2EB324F08BF93
:1062D000012043E80212002AE8D1704730B4044696
:1062E00054E8000F0D4644E80053002BF8D1156028
:1062F00030BC704730B4044654E8000F40EA010552
:1063000044E80053002BF7D1156030BC704730B41F
:10631000044654E8000F00EA010544E80053002B4E
:10632000F7D1156030BC704730B4044654E8000F14
:1063300080EA010544E80053002BF7D1156030BC1A
:10634000704730B4044654E8000F00EB010544E800
:106350000053002BF7D1156030BC704730B40446B1
:1063600054E8000FA0EB010544E80053002BF7D1DF
:10637000156030BC704770B404464FF0000054E81C
:10638000006F0D68AE4207BF44E80023012044E8D7
:1063900000630E60002B1CBF0020F0E770BC70474C
:1063A00030B4044654E8000F88422CBF451A054615
:1063B00044E80053002BF5D1156030BC7047000055
:1063C0000648804706480047FEE7FEE7FEE7FEE78F
:1063D000FEE7FEE7FEE7FEE7FEE7FEE731680200C4
:1063E000016202002DE9F05F0546002092469B46BF
:1063F00088460646814640241BE0284641464746DB
:10640000224600F079F853465A46C01A914110D3FB
:1064100011461846224600F016F82D1A67EB0108BF
:106420004F4622460120002100F00DF817EB00092D
:106430004E41201EA4F10104DFDC484631462A46C5
:106440004346BDE8F09F202A04DB203A00FA02F11F
:10645000002070479140C2F1200320FA03F3194352
:1064600090407047004870470404030010B5431A79
:10647000934209D28318881803E010F8011D03F82D
:10648000011D521EF9D210BD40EA01039B0703D043
:1064900009E008C9121F08C0042AFAD203E011F863
:1064A000013B00F8013B521EF9D210BDD2B201E00F
:1064B00000F8012B491EFBD270470022F6E710B509
:1064C00013460A4604461946FFF7F0FF204610BD62
:1064D000421C10F8011B0029FBD1801A704730B50F
:1064E00004460020034600E05B1C934203D2E05CBC
:1064F000CD5C401BF8D030BD202A04DB203A21FAC5
:1065000002F00021704721FA02F3D040C2F12002CC
:106510009140084319467047064C074D06E0E06875
:1065200040F0010394E8070098471034AC42F6D3DA
:10653000FFF76AFED80B0300F80B030070B58C1848
:1065400010F8015B15F0070301D110F8013B2A1187
:1065500006D110F8012B03E010F8016B01F8016B74
:106560005B1EF9D12B0705D40023521E0DD401F870
:10657000013BFAE710F8013BCB1A921C03E013F839
:10658000015B01F8015B521EF9D5A142D8D300206E
:1065900070BD00002DE9F04F00268DB0DFF8A0811E
:1065A000B14604964FF48075012437460596284677
:1065B00005F052FA38B1D8F80403204203D0284637
:1065C00005F040FA26432D1D64007F1CADB2082F54
:1065D000EDD34FF4BE74204605F03EFA48B1204694
:1065E00005F030FA46F0004604AA0221002005F02A
:1065F00013FA544C16F0FF0F15D00127002537422F
:106600000DD008EB8501D1F81005D1F81015C0F3B5
:10661000052054F82520C1F3014102B190477F00C5
:106620006D1C082DEBD3002E7EDA0020CDF82890CB
:10663000411E0DF1100B07AACDF82C9042F8201046
:10664000401C91460228F9D300252E46A11911F8C5
:10665000607F91F9000027F0C008401C40D007A9D6
:10666000404604F0A4FB40B34FEA971A404602F0BC
:10667000DBF854F820701FB1BAF1030F03D006E025
:10668000BAF1030F2CD10AA9404604F098FB02A8E6
:10669000CDF8088005F064F9029900EB8100D0F88C
:1066A000000704A9C0F301400290404604F07FFBBC
:1066B0000028029802D0022802D011E003280FD14E
:1066C000BAF1030F08D10298022833D002214046C4
:1066D00005F020F96D1CEDB217B151464046B847A0
:1066E000761C042EB2D3002D21D001AA0221002055
:1066F00005F092F900205A460DF1040152F820608D
:1067000051F82030B34217D000200AAE4FEA0903F7
:1067100051F8207042F8207056F8207043F820702D
:10672000401C0228F4D300E001E0002D8CD10DB014
:10673000BDE8F08F0321CAE7401C0228DED3F6E74C
:10674000006000409833002000F01F0201219140BA
:106750004009800000F1E020C0F88012704700F08E
:106760001F02012191404009800000F1E020C0F8A3
:106770000011704700F01F02012191404009800084
:1067800000F1E020C0F8001270474907090E002808
:1067900006DA00F00F0000F1E02080F8141D7047C9
:1067A00000F1E02080F800147047000070B54FF44D
:1067B0008076304604F03AFC114CB50560B13046A5
:1067C00004F03BFC0120C5F80803607920B90120E2
:1067D00060712168002088474FF48276304604F0CB
:1067E00025FC00280AD0304604F027FC0220C5F81A
:1067F00008032168BDE870400120084770BD000013
:10680000882C002007480021C0F84011C0F844112E
:10681000C0F84811C0F84C11C0F80011C0F80411BC
:1068200008F008BE0010014008F052BD05F0ACBEF3
:1068300030B54FF0805000228300D0F83011C3F8FB
:106840000C21C3F81021624B1A60624B1B68624C2A
:106850002360604B1B1D1B68241D23605D4B0833A8
:106860001B68241D23605B4B0C331B68241D2360B5
:10687000584B10331B68241D2360564B14331B6880
:10688000241D2360534B18331B68534C2034236062
:10689000504B1C331B68241D23604E4B20331B6858
:1068A000241D23604B4B24331B68241D2360494B5C
:1068B00028331B68241D2360464B2C331B68241D82
:1068C0002360444B30331B68434C40342360414BBE
:1068D00034331B68241D23603E4B38331B68241D52
:1068E00023603C4B3C331B68241D2360394B4033F1
:1068F0001B68241D23600124082902D1D0F83431FB
:1069000013B1082904D006E0354B3449196005E07D
:10691000D0F8343113B1082904D006E0314BFB2103
:10692000196005E0D0F8343113B1082908D00EE021
:1069300090F858322C48016863F30301016002E0CB
:10694000D0F834311BB929494FF400700860284849
:106950000168C90702D06FF0010101602548016894
:1069600041F470010160BFF34F8FBFF36F8F4FF0A1
:106970001021D1F80002002803DBD1F8040200281E
:1069800022DA1D4B1C601D480468002CFCD0122428
:10699000C1F800420568002DFCD0C1F8044201682E
:1069A0000029FCD01A6001680029FCD0BFF34F8F8A
:1069B00010487C380168124A01F4E061114301601B
:1069C000BFF34F8F00BFFDE70F490E48086030BD91
:1069D000380500400404001020C500404881030031
:1069E0008C56004018F50040E40E004040960240EE
:1069F0000004004088ED00E004E5014000E40140AF
:106A00000400FA050090D003AC2D00200148006876
:106A100000470000902C002002E008C8121F08C1A7
:106A2000002AFAD170477047002001E001C1121F0F
:106A3000002AFBD1704700000121202803DA8140A1
:106A40000548014003E0402802DA2038814009B1BE
:106A50000120704700207047FC06FFBD10B560B1F3
:106A600059B102780B785208B2EB530F05D10622C8
:106A7000401C491CFFF733FD08B1002010BD012068
:106A800010BD800701D00020704701207047C36807
:106A90008B4206D811440069491E814201D8012069
:106AA00070470020704710B501220221002001F03C
:106AB000CBFC08B1072810D107220221012001F0E8
:106AC000C3FC08B1072808D100210A22084601F0BA
:106AD000BBFC08B1072800D1002010BD10B550B193
:106AE0000A480321008801EB004009A105F0A4F940
:106AF00007F0C2F903E00321094800F055FD002822
:106B000003D0BDE8104000F0CBB810BDF82D002038
:106B1000457261736520626F6E647321000000002E
:106B20000C2F002070B58CB015460E4600236C4625
:106B3000C3F10F01415CE1545B1C102BF8D30D2114
:106B400004F11000FFF7B9FC0020C0F10F02315C26
:106B50002244401C11740328F7D3684646DF002006
:106B6000C0F10F01214491F820102954401C032842
:106B7000F6D30CB070BD022001F068BB0149097961
:106B800000F066BF0C2C002070B50024064D06E016
:106B90006868012110F8340005F0E0FD641C2878D5
:106BA0008442F5D3002070BD982C0020F8B515461E
:106BB0000C460646052A01D20720F8BD05F0C6FEA0
:106BC00018B905F089FE0028F7D1124900224E605D
:106BD0000C708D60C1E90422C1E906220E4D0DE062
:106BE00006EBC4002968009181788DF801100078C7
:106BF0000A4A694605F0FEFD0028DED1641EE4B2B3
:106C0000EED2BDE8F84004480021054A001D00F01E
:106C100053B80000982C00207C00030071990200FA
:106C2000158D020072B605F0BDF900BF04F0F4FF47
:106C30000028FBD1104C0121208801EB00400FA15E
:106C400005F0FAF810480068C00700D000BE2088A0
:106C5000022101EB00400DA105F0EEF8BFF34F8FCC
:106C60000948E43801680D4A01F4E061114301600C
:106C7000BFF34F8F00BFFDE7F82D00204661746120
:106C80006C206572726F7200F0ED00E053797374DE
:106C9000656D207265736574000000000400FA05DC
:106CA0000EB500210091CDE901106A4644F20100C1
:106CB000FFF7B8FF0EBD0000074B9B7823B12AB148
:106CC00020B10068037C1BB1082070470720704783
:106CD00041744261002070477434002070B507F0A1
:106CE0001BFC104800240B21047044700E4D817071
:106CF00014206C602C706C70FFF726FD07211420A7
:106D0000FFF743FD1420FFF72AFD08480460072120
:106D10001120FFF73AFD0548001F0068A860002019
:106D200070BD000074340020B82C0020081501400C
:106D30002DE9FC47DFF8789099F8023073B368B317
:106D4000052902D20720BDE8FC87436933B3437CA1
:106D5000012B25D0002704460025884616468DF8CD
:106D60000050684600F038F801A808F031FEC8B1BC
:106D7000012101700F4944600968C0E90218C0E9A7
:106D800004769DF8040089F801009DF8000000F0E9
:106D900047F81420FFF7EEFC2846D4E70820D2E796
:106DA0000F46D8E704259DF8000000F039F8F3E716
:106DB00074340020041501400649897839B130B196
:106DC000416921B100210174022108F00FBB0820A4
:106DD000704700007434002030B5EFF3108172B6B4
:106DE0000D4A9468012324B10370002900D162B6D2
:106DF00030BD93604FF0E023D3F88051074C25401D
:106E00001560C3F88041D3F8844154605A17C3F821
:106E1000842100220270E8E780350020FC06FFBDD7
:106E20000B498A68002A11D000280FD1EFF3108097
:106E300072B60B684FF0E022C2F800314B68C2F81E
:106E4000043100228A60002800D162B67047000039
:106E50008035002010B5144C00224FF4803120689A
:106E6000FFF766FF08B1FFF71BFF00224FF4004158
:106E70006068FFF75DFF08B1FFF712FF002242F2E2
:106E80006661A068FFF754FF08B1FFF709FF002211
:106E90004FF42031E068FFF74BFF002803D0BDE836
:106EA0001040FFF7FDBE10BD10FF020070B5054693
:106EB00008680C46411C04D004F087FD206804F0EB
:106EC00015FD6068411C02D0002104F0FDFC29681A
:106ED000A069C1F82405607D227D29681043C1F8AE
:106EE0006C05D4E900122868C0F81425C0F80C1508
:106EF000207D012814D1A068411C02D0002104F09B
:106F0000E3FCE068411C04D004F05FFDE06804F09D
:106F1000EDFCD4E902122868C0F80825C0F8101565
:106F200070BD70B5054608680C46411C04D004F0DD
:106F300056FD206804F0E4FC6068411C02D000218A
:106F400004F0CBFC2968A069C1F82405607D217D8F
:106F50002A680843C2F86C05D4E900122868C0F812
:106F60000C15C0F81425207D012814D1A068411CFF
:106F700002D0002104F0B1FCE068411C04D004F010
:106F80002EFDE06804F0BCFCD4E902122868C0F8C9
:106F90000825C0F8101570BD03F056BB2DE9F04769
:106FA000074600888EB0804603F042F882460446C9
:106FB0002D4800252A460178404600F061FD787989
:106FC000400734D501254FF6FF7603AB2A4607214B
:106FD000504606F0ABF9010004D0404607F094FC9F
:106FE00000252BE0B1463146049802F075FF0646B5
:106FF00048450FD004460146404603F003F840469A
:10700000FFF7BCFD30B9404607F050FC4046FFF7A3
:10701000B5FD48B122460721504606F0FDF90100B2
:1070200003D0404607F070FC00254E4506D0404690
:1070300006F060FB10B1504602F0E6FF02208DF82A
:107040001800ADF81A807879400701D5012000E0DA
:1070500002208DF820008DF8215006A801F0CEFF07
:107060000EB0BDE8F08700000C2C00202DE9F043A5
:107070000546407C93B00E460024A0B107949DF8CD
:107080001C0020F00F00401C20F0F00010308DF8A4
:107090001C00707B8DF81D009DF81E0020F006007E
:1070A000801C8DF81E001C216846FFF706FA9DF82B
:1070B000000040F002008DF80000697C11B140F042
:1070C000100001E020F010008DF8000001940394FE
:1070D0000494687C00B107A8CDE9050401278DF868
:1070E000427042F61920ADF840000D94B07B8DF847
:1070F0003400F07B8DF835009DF83600142120F027
:107100000600801C20F019008DF83600307B8DF8C9
:10711000440008A8FFF7D1F90DF140080DF134093A
:10712000ADF8287011A8CDE90889ADF82A40ADF86E
:107130002C700C90A888AB1D08AA6946AADF00280D
:1071400038D1B06898B38DF8427042F60810ADF8A7
:1071500040000D94307C8DF834009DF8350020F00F
:10716000FF008DF835009DF8360020F00600801CE9
:1071700020F019008DF836000EA8B16800F0D8FF95
:107180000646142108A8FFF798F9ADF828600EA864
:10719000CDE90889ADF82A40ADF82C600C90E8885C
:1071A00005F10E0208A9ABDF002803D101E0FFE7DB
:1071B000EC81002013B0BDE8F083000010B50E494B
:1071C0000E4807F018FCC1B20B484FF6FE72EC38BF
:1071D00000F006FB00280DD008280BD0132809D09A
:1071E000112807D043F20141884203D0BDE8104086
:1071F000FFF756BD10BD0000C42F0020902B0020CB
:107200000A4601461046AEDF70472DE9FC470025CF
:1072100017880646158090F82D001446894630B12F
:107220003A462146484600F055FC051E09D1B07883
:107230004FF00C0A18B32088C846001DB84202D986
:107240005046BDE8FC87684679DF0028F9D12088E0
:10725000032108F8001020881921401C80B22080EA
:1072600008F800102088401C80B2208000EB080144
:10727000BDF8000008F0DAFA218808442080F07890
:107280000222C8B1218896F9033001F1030C484667
:10729000BC45D5D8425421884FF0010C491C89B215
:1072A000218000F801C02188491C89B2218009F899
:1072B00001302088401C20807068B8B1218890F986
:1072C000003001F1030C4846BC45B9D8425421882E
:1072D0000A22491C89B2218042542188491C89B262
:1072E000218009F801302088401C2080308950B16D
:1072F000CDE900474B460622022106F1080008F0BE
:107300007FFB051E9DD1308A50B1CDE900474B4629
:107310000722032106F1100008F072FB051E90D130
:10732000308B50B1CDE900474B461522142106F1B0
:10733000180008F065FB051E83D1306A30B13B466A
:107340002246494601F07BFB051EDBD1706A30B155
:107350003B462246494603F0E5FA051ED2D196F88F
:107360002C0038B13B4622464946304607F0E2FB46
:10737000051EC7D1307838B13B46224649463046D3
:1073800003F056FB051EBDD128465AE718B5044642
:107390000020ADF8000013466A46204600F006F8CB
:1073A000002802D0BDF80000204418BD70B588B197
:1073B00082B10024158803E0065D641C3444A4B245
:1073C000A54203D8061976789E4201D08C42F3D3A9
:1073D0008C4201D3002070BDA11C1180005D401EB5
:1073E00080B270BD80F8301070472DE9F0410E007A
:1073F000044606D02CB196F87A000025012803D067
:1074000006E00E20BDE8F08196F89800012821D012
:107410004FF00108A5702C2206F17801201DFFF71E
:1074200025F884F83050D6F8A4006063D6F8A80098
:10743000A0634FF6FF70A4F8A80004F19400C4F80C
:10744000A400C4F8AA50A4F8AE5084F8B050207834
:1074500010B104E00720D5E7FF2084F8540004F1C0
:1074600055011F27C4F89410A4F8987004F19802ED
:107470003046FFF7CAFE0028C4D116F13C0F0ED0EB
:1074800004F17401C4F89C10A4F8A07004F1A002E7
:1074900006F13C00FFF7B9FE0028B3D103E0C4F8C1
:1074A0009C50A4F8A05084F85180208BA4F8480088
:1074B00084F83C80256484F85050606960644646D6
:1074C00004F13C02002104F1540072DF002899D13C
:1074D000267097E710B50288102A1BD0112A20D0F9
:1074E000262A1DD1007A0C46012801D0022817D186
:1074F000A0780521401CB0FBF1F201FB12012046EF
:1075000000F052F800280BD0A16B002908D0BDE88C
:1075100010400847C27B012A02D18088A1F8A80048
:1075200010BD0C46002184F8B2108088B4F8A81071
:107530008842F5D120790028F2D10121DFE710B58A
:107540000C46022801D0032810D1607800280DD005
:1075500000206070A178204600F026F8002805D0B1
:10756000A16B002902D0BDE81040084710BD10B53E
:10757000044690F8540074DF012084F8B200002023
:1075800084F8B40084F850000621204601F03EFF44
:10759000002808D1A178204600F006F810B1A16BB0
:1075A00001B18847002010BD2DE9F05F0446007846
:1075B0000F4638B1A770002003F090FF012620B1DC
:1075C000667007E10820BDE8F09F0025C4F8AA50C6
:1075D000A4F8AE5084F8B050A07910B1A07801287A
:1075E00006D0E07968B1A078012801D0022808D13E
:1075F000616B21B184F8B1600820884701E084F80C
:10760000B15004F1AB0100200A5C0AB1304603E03E
:10761000401C0628F8D300204FF002084FF0030B5F
:10762000012F06D0022F0CD0032F0FD0042F15D11D
:1076300010E0A17929B194F8241011B908B13046AD
:107640000DE0E17911B108B1404608E0207A08B1B7
:10765000584604E0607A08B1042000E02846A07093
:10766000616B41B1032801D0042804D1607910B1C5
:1076700094F8B200A0B184F8B35004F13C00182192
:107680000746FEF71AFF04F12C0084F83C6081469F
:1076900006F064F958B194F82C0084F8510008E021
:1076A00084F8B45084F8B36007208847E5E784F88D
:1076B000516094F8240050B1484606F04FF920B1CB
:1076C00094F8280084F8520001E084F8526084F8AD
:1076D0005050A27804F1AA0104F194094FF0060A6F
:1076E000052A60D2DFE802F078030F223F0084F819
:1076F0003160C4F8A450C4E9101584F83C8080209F
:10770000A4F8480051E084F8318094F824203846E9
:1077100012B10722027001E080F800B0228A828153
:10772000C4F8A4504160E168B9603EE06069B860A7
:10773000208BB88194F824003D4610B184F83CA019
:1077400001E084F83C60204608F01EF940B185F85D
:1077500014800421204601F059FE20BB05211EE0C3
:1077600084F831B01DE0E069B860208CB88194F8ED
:1077700024003D4610B184F83CA001E084F83C6050
:10778000204608F001F948B185F81480042120460C
:1077900001F03CFE38B984F831A002E0042184F8FD
:1077A0003110C4F8A490A07878B13A4604F154009E
:1077B000D4F8A41072DF00287FF405AF94F83010DD
:1077C00094F8540073DF0028F6D1616B11B194F87E
:1077D000310088470020F6E684F83150F5E70000D4
:1077E000F7B594B0174605003CD0287C9DF854109E
:1077F0000024884252D000264FF0010E0D9615A8A5
:10780000ADF834E00E90ADF83660E9880DAA4FF679
:10781000FF70ACDF040026D19DF854002874687C0A
:10782000A0B30F96109611961296E888ADF83C001A
:10783000BDF83600ADF840000DA811900E981290DA
:10784000A7F57F408DF83EE0FE3805D039460FA8F9
:10785000FFF7D6FC044621E0684600F09DF80025BD
:107860006F460FE00E2017B0F0BD00BF07EB4506D6
:10787000B08800F0CFF8022803D144B10FA9B08836
:10788000AEDF6D1C0098A842F0D807E005E0B18893
:107890000FA8FFF7B5FC0446F3E708242046E2E70B
:1078A00038B50D46040018D0BDB12868206028798D
:1078B0006074FF20207401208DF8020041F60F0053
:1078C000ADF80000221D69460120A8DF002803D181
:1078D00029462046FFF7CAFB38BD0E2038BD38B513
:1078E000002924D0002822D00288502A1FD1054622
:1078F000487C0C4600281AD0E9886289A81D91426C
:1079000015D14189022912D1216800290FD00C30EC
:1079100000F00AFC08B1002000E001208DF8000012
:10792000A888ADF80200226869462046904738BD15
:1079300070B5040012D001461C221448FEF796FDD3
:107940001248134D0560206850B17ADF002806D137
:107950002068016829604068686005E00E2070BDFD
:107960000B487BDF0028FAD108484FF6FF71143826
:10797000084A20F8041B0549343901600021FFF74B
:107980009BF90028EBD0032070BD0000943000204C
:10799000CC2B002021F902000149496801F030B8E0
:1079A000B030002010B5044600F08AF8002805D059
:1079B0002146BDE81040024803F05DB910BD00004B
:1079C000C030002070B515460E46044607F0E8FFAB
:1079D000002809D0054800EB840080692A4631461A
:1079E000BDE8704001F050BD70BD0000B030002017
:1079F00070B50546002400F063F838B12946044804
:107A000003F039F908B1022400E00124204670BDDA
:107A1000BC30002070B50546002400F051F838B1A4
:107A20002946044803F027F908B1022400E00124A4
:107A3000204670BDB830002010B51821034803F06F
:107A4000F5F8182800D0C0B210BD0000B0300020FA
:107A500070B505460C46084607F0A2FF60B12846FF
:107A600000F02EF840B10548294600EB8400BDE83F
:107A70007040183003F0FFB8002070BDB030002017
:107A800070B5054614460E46084607F089FF0028E3
:107A900012D0284600F014F800280DD007482946D7
:107AA00000EB860018301CB1BDE8704003F0EEB862
:107AB000BDE8704003F09FB870BD0000B0300020FA
:107AC000142801D3002070470146014803F0D3B8C1
:107AD000B43000207CB5054608880C460930904239
:107AE00001D90C207CBD68466DDF0028FAD12188C1
:107AF0000820685420881B21401C80B22080295413
:107B00002088401C80B220802844DDF801100160EC
:107B1000BDF8051081802088801D80B220809DF8EE
:107B20000010490800D0012129542088401C2080E1
:107B300000207CBD7FB5044601208DF8060041F68B
:107B40000A00ADF80400454A01A90120A8DF002879
:107B50007ED1228804F13C0552B140482B46801C5E
:107B6000009042F62920616800F066FE002873D17B
:107B7000228952B139482B460A30009042F624201F
:107B8000E16800F059FE002866D1228A52B13348DC
:107B90002B461230009042F62520616900F04CFE21
:107BA000002859D1228B52B12C482B461A30009014
:107BB00042F62720E16900F03FFE00284CD1228CDC
:107BC00052B126482B462230009042F62620616AA8
:107BD00000F032FE00283FD1228D52B11F482B46C3
:107BE0002A30009042F62820E16A00F025FE0028A5
:107BF00032D1216B71B102A807F048FB17482B4620
:107C000032300090082202A942F6232000F014FE30
:107C1000002821D1606B58B110492B463A310091B0
:107C20000279016842F62A2000F006FE002813D1EE
:107C3000A16B81B102A806F078F908482B464230C2
:107C40000090072202A942F6502000F0F5FD00E066
:107C500002E0002800D1002004B070BD2A2C0020D2
:107C600038B502880446212A2FD012DC1E484FF076
:107C700003011E4D0088102A01EB004011D0112A8B
:107C800006D1227A1AA104F0DBF84FF6FF70688063
:107C900038BD3B2A23D0562AFAD18088132176DFBB
:107CA0000DE01AA104F0C8F8072000F0EFFB08B1BE
:107CB000FEF7F6FFA1886980174803F03FF9002816
:107CC000E6D0BDE83840FEF7EBBF00200090A0886A
:107CD00069468FDF0028DBD0FEF7E2FF38BD8088E1
:107CE000132176DFEBE70000F82D0020882B002021
:107CF000446973636F6E6E65637465642C2072658E
:107D000061736F6E2025642E00000000436F6E6E5D
:107D100065637465642E0000002F002010B51A4CB6
:107D20000188606810290ED011292BD1401E606097
:107D300028D1FEF7B8FE002824D02168002921D0E0
:107D4000BDE810400847D0B900210122084600F0E4
:107D50007BFB08B107280FD107220221012000F088
:107D600073FB08B1072807D104220221002000F08C
:107D70006BFB20B1072802D0216801B188476068F9
:107D8000401C606010BD0000C42B00202DE9F047AE
:107D900001883B4E40F2F3194FF6FF7510291BD0B6
:107DA00011293ED0122954D0502946D1C188F289D8
:107DB000841D914241D1618902293ED18688304695
:107DC00002F0E2F9050038D004F10C0000F0ACF943
:107DD000A8B3294630464EE0C17B87880446012976
:107DE0002BD1A846284602F0CFF9050017D02F80E6
:107DF00000202872234843464A460168C5F80A1005
:107E00004068C5F80E0004F1100105F10A0002F007
:107E100087FA6872F08900280FD129462AE00420E9
:107E200013E0808802F0B0F9040006D06068FEF725
:107E3000C3FF08B106F04CFD2580BDE8F087FFE7E1
:107E40006868FEF7B9FF0028F7D0BDE8F04706F0F4
:107E50003FBD87880646384602F096F90400ECD00C
:107E60002B464A4606F1080104F10A0002F058FACE
:107E7000607221463846BDE8F04700F027BE00009A
:107E800094300020CC2B00202DE9F04F0746858848
:107E900002883D48012197B08346102A09D0112A53
:107EA00049D01A2A6CD1387AB1EB101F45D2012281
:107EB00044E0354C083CA068C0430B9061680BA8B7
:107EC00002F0FDFE0B990CA800F09AFD2C220CA9E3
:107ED0006846FEF7CBFA0026E946A04610E000BF50
:107EE00009EB46005FF00004B0F804A008EB840042
:107EF0005146001D02F07FFE641C1D2CF6D3761C3B
:107F00000098B042ECD8142D05D317B00420BDE87A
:107F1000F04FFEF7C5BE2946584602F0B7FE294687
:107F200008F1040002F0B2FEF87B012828D01648C0
:107F30002946001D15E029461AE000220221B1EB76
:107F4000101F01D2012600E000260F49083901F177
:107F50001000041D294682B102F098FE36B1294670
:107F6000204617B0BDE8F04F02F090BE29462046EB
:107F700017B0BDE8F04F02F03EBE02F03CFEF5E760
:107F800017B0BDE8F08F0000B830002010B50446EF
:107F90000748007800280AD0204601F023FF204639
:107FA00006F0CEFE2046BDE8104001F0E3BB10BD58
:107FB000FC2B002030B50446008CC3B0A0F57F42F6
:107FC000FF3A23D06A46204601F084FE0546ADF80C
:107FD000F40000203E903F90409041902189ADF800
:107FE000F8100121ADF8FC008DF8FA103DA8409082
:107FF000CDF804D1208C3EA9AEDF002804D1BDF815
:10800000F410A94200D00C2043B030BD0820FBE79B
:1080100038B5044608682060087960714FF6FF7033
:108020002084002084F82200A4F84C00F42084F876
:108030004E0001208DF8020041F60D000D46ADF80E
:108040000000A21D69460120A8DF00280ED12946A4
:10805000204601F0DDFD002808D1A86828B1294696
:10806000204600F06BF8002800D1002038BD38B55C
:108070000288102A15D0112A15D0502A16D130F8AE
:10808000062F8B899A4211D10C46418902290DD1C4
:10809000216800290AD00C3000F046F838B10020E1
:1080A00006E0808801E04FF6FF70088438BD0120AB
:1080B0008DF80000226869462046904738BD028C42
:1080C0004B889A4208D10A88A2F52063773B03D1F6
:1080D0000979C91E80F84E10704770B50446B0F893
:1080E0004C000D4614280AD104F126012622881ED0
:1080F000FEF7BCF9B4F84C00401EA4F84C00B4F8EC
:108100004C0004EB4001401CA4F84C008D8470BD71
:1081100080F82210704770B504460D460846FEF7F9
:10812000D7F92080656070BD007800F001007047CD
:108130000A7802704978417002207047F0B58FB01C
:108140000D4606461C216846FEF7B7F900249DF847
:108150000000039440F002008DF800000127019414
:108160008DF8367042F63820049405940694ADF8E4
:1081700034000C94E87B8DF83000287C8DF83100B9
:108180009DF83200142120F00600801C20F0190018
:108190008DF8320007A8FEF790F90DA807900CA8FB
:1081A000ADF824700890ADF82640ADF82870A868A6
:1081B0000B90F08806F1100307AA6946AADF0FB0FA
:1081C000F0BD00000149085C7047000024FF020078
:1081D000084908B5085C0090684603F0B3FBD0F886
:1081E00010050099C84010F0010000D0012080F077
:1081F000010008BD24FF02002DE9FC410646C0072E
:108200004FF000050ED0104F00240122385D00957C
:1082100000231146019503F0E1FA641C042CF4D309
:1082200000F04EF8B0070DD5074E0024361D002291
:10823000305D032300951146019503F0CFFA641CCD
:10824000042CF4D3BDE8FC8120FF0200094908B5E5
:10825000085C0090684603F075FBD0F80425009B8D
:108260000121994021EA0203C0F808351140C0F805
:108270000C1508BD20FF02000249085C012103F033
:10828000B8BB000020FF02000249085C002103F097
:10829000B0BB000020FF0200084908B5085C009050
:1082A000684603F04FFBD0F804050099C84010F071
:1082B000010000D0012080F0010008BD20FF020075
:1082C00010B500242046FFF7D7FF641C042CF9D317
:1082D00010BD10B500242046FFF7D6FF641C042C07
:1082E000F9D310BD10B50246064B4FF0FF30002108
:1082F0005C5C944201D1084610BD491C0429F7D3A7
:1083000010BD000024FF020070B50C4E0C004FF0B1
:10831000000530600BD0012000F06AF808B102209F
:1083200004E0002000F064F800B10B2020707068B9
:1083300010B9FEF7B8FB0546284670BDC42B0020D7
:1083400010B5002000F0D4F908B1062806D10120AC
:1083500000F0CEF908B1062800D1002010BD0000C1
:108360002DE9F0470D468146FFF7BCFF044604287F
:1083700036D2DFF874801B481C4EA8F10C0725B3D9
:10838000012D0ED0022D2BD104EB44003044457852
:10839000002D25D0B968002922D02846BDE8F04735
:1083A000084704EB4401755C0E44717849B10E4AEC
:1083B0004FF40041093A8068FEF7BAFC08B987F823
:1083C0000390B17808F80410E2E78068FEF7F4FC47
:1083D00004EB4401314418F804008D78A842D7D04A
:1083E000BDE8F08728FF0200C02B002034300020B9
:1083F000042801D2FFF7ECBE002070470146104868
:1084000010B54088042907D007290ED00A2915D1B4
:10841000BDE8104006F080BC132176DF0CE0002898
:108420000CD0BDE81040FEF73BBCA0F57F41FF3902
:1084300004D10448FFF79BF80828F0D110BD0000D4
:10844000882B00200C2F002070B50023042810D2A8
:108450000D4D00EB4004012A02D101290CD000226D
:10846000094E00EB4000304461B1012906D00229D9
:1084700006D00723184670BD0E30C2B22A55F9E760
:108480004270F7E78270F5E734300020044A014675
:1084900000201279D20702D0084600F04DB870478C
:1084A000B42B002070B506461E480024C0E90161C7
:1084B000B00720D50025012211462846FFF7C4FF4A
:1084C0006D1C0446042D02D2002CF4D013E094B9A4
:1084D00040F2666204211448FEF768FB04000AD1EA
:1084E000FEF752FB040006D10F48104A0021001F7E
:1084F000FEF7E2FB0446F00712D00120FFF77CFEF6
:1085000074B909480A4A00210C38FEF7D5FB04006B
:1085100006D10548074A01210838FEF7CDFB04467D
:10852000204670BDB42B002034FF0200BD8702003E
:10853000B5A30200776B02002DE9F05F6A4C054697
:1085400000266078B34618B184F801B001F01AFF34
:10855000664F4FF47A694FF4C87A4FF00108182D2E
:1085600062D2DFE805F0AC0C0C31404D62676B74F1
:108570006B74BE7D7D7D7D7DACAFB2B5BEBE00208F
:10858000FFF78AFE00284FF0000008D0FFF774FEC6
:10859000022D02D14FF4E16008E0484606E0FFF703
:1085A00073FE022D01D1C82000E05046410CC003EB
:1085B0004FF4FA72801841F1000125705200002337
:1085C000FDF710FF01462AE00020FFF765FE0028B6
:1085D0004FF0000004D0FFF74FFE4FF44870E5E77E
:1085E000FFF752FEDFE70020FFF756FE00284FF0AE
:1085F000000002D0FFF740FECFE7FFF745FED4E7CB
:108600000020FFF749FE00284FF0000002D0FFF7DE
:1086100033FE01E0FFF738FE257041F69A11002283
:108620003868FEF785FB064646E00020FFF70EFEA1
:10863000257008E0002051E025703DE084F80180BD
:108640000120FFF703FE002240F6CD41E8E784F861
:1086500001800120FFF7FAFD00224FF48041DFE79F
:108660007868FEF7A9FB0646D5F1110000D02EB1BF
:108670000220FFF701FE84F802B01DE0012816D9A0
:1086800080B2C8214843C117C90341EA5041C00321
:108690004FF4FA72801841F1000152000023FDF7F7
:1086A000A1FE014600227868FEF742FB0646022042
:1086B000FFF7EAFD84F802803046BDE8F09F01F044
:1086C00061FEB9E701F05EFEB4E701F05BFE04E095
:1086D00001F058FE0020FFF7D7FD0120FFF7D4FD81
:1086E000AAE7FFF7F6FDA7E7B42B002028FF02005A
:1086F000012107F0EDB900002DE9F8430546861C7D
:1087000000208DF8000090460F464FF001096846A2
:10871000FEF762FB1B4C20683860D4E90001401A68
:10872000A16804F21C47081A0EE00121384602F045
:10873000C0FA01F0DFFF0146384602F0BAFAD4E988
:108740000001401AA168081A401C8642EDD8B8F111
:10875000000F03D0052065F3891002E0062065F3C1
:108760009F50A2682168114004EB8101C860206815
:10877000304420609DF80000FEF752FB4846BDE8FB
:10878000F88300001838002030B482680468531C55
:108790008360A154D0E901128A4202D330BC02F0B6
:1087A000CABC30BC70470000034803C8814201D1F5
:1087B00001207047002070471838002000780221FF
:1087C000FFF7CEBD05494FF0FF32082841F82020C1
:1087D00002D3084480F858207047000098330020E6
:1087E000F0B54FF0FF3512B10023082601E0082351
:1087F0000C260C4C05E000BF54F823707F1C04D0FD
:108800005B1CB342F8D32846F0BD26185DB286F84B
:10881000305044F82310002AF5D1E11881F85800AF
:10882000F1E70000983300200249084490F9300035
:1088300070470000983300202DE9F0438FB01E46AA
:10884000DDF8589015460F00804602D10020FEF753
:1088500027FA15B90020FEF723FA1C216846FDF718
:108860002CFE00249DF80000039440F002008DF8D7
:108870000000012001948DF83600049405940694BC
:10888000ADF834800C9430788DF8300070788DF825
:1088900031009DF83200142120F00600801C20F0E9
:1088A00019008DF8320007A8FDF707FE0DA8079004
:1088B0000CA808900748ADF82450ADF82640ADF854
:1088C00028500B974B4607AA69460088AADF0FB0CD
:1088D000BDE8F0832A2C002070B504464FF6FF75E2
:1088E0000A462846AC4208D14FF48074214610460F
:1088F00005F08CF9A04209D070BDFF2CFCD82146B0
:10890000104605F076F908B1204670BD284670BDC6
:1089100070B5084C050009D010342168002907D033
:1089200008682060496828468847F6E70834F4E775
:1089300070BD000084330020054A012120B10128C8
:1089400005D19170FFF7E4BF51700020FAE770473E
:10895000843300202DE9F05F26484168F1B3DFF849
:1089600098B00E688146DBF8004087688078E11B8C
:1089700021F07F45ED1CB0B9DFF880804FF48030E6
:10898000C8F84403C8F804031120FDF7DDFE1120E8
:10899000FDF7E5FE4FF0010AC8F800A02F2003F014
:1089A000D5FE89F802A0B54200D23546124BE8192F
:1089B0003C3320F07F401860DBF800105A46091B5A
:1089C00021F07F41001B20F07F40C91C81420FD95C
:1089D000106818602F2003F0B9FE00E004E0BDE845
:1089E000F05F1120FDF7C6BEBDE8F05F05F094BD55
:1089F000BDE8F09FB82C0020041501400010014094
:108A000073B58CB00646002000900D9880B100240C
:108A10006D4621460DA802F02EF930B1009805EB05
:108A2000400084800098401C0090641C142CF0D3FB
:108A30002C2269463046FDF719FD0EB070BD2DE9B8
:108A4000F04117880646B81D14460D46984202D9D3
:108A50000C20BDE8F0813188072206290AD34FF4A3
:108A6000486C4FF6FF73614501D9994202D1708875
:108A7000062801D21046ECE7604501D99842F9D1A9
:108A8000994203D0984201D08142F3D80520E8559D
:108A900020881221401C80B2208029542088401C4C
:108AA00080B220804119308806F0C0FE2188084439
:108AB00080B220804119708806F0B8FE21880844F1
:108AC00020800020C5E7FEF7EBB8000038B54A7AF1
:108AD0000F4B62B100220A725969002906D00122A7
:108AE0008DF80020ADF802006846884738BD0A7A44
:108AF00062B19B684C68024619462046FEF718F999
:108B00000028F3D0BDE8384005F0E2BE5B68F1E72D
:108B100094300020F0B585B016460F4604461D4639
:108B200014220B496846FDF7A1FC0A488DF808702D
:108B3000ADF80240ADF80A608DF80C5001780022C3
:108B40002046FEF79DFF684600F058FA05B0F0BDDC
:108B5000400003000C2C0020F0B587B00746002031
:108B60000490ADF810100590ADF81210019002902D
:108B700001AA04A9384690DF060022D003F08CFD3C
:108B8000114C0346012520883A4605EB00400F4969
:108B900003F05DF9BDF8042012B9BDF8060038B144
:108BA0002088BDF8063005EB004009A103F04FF91D
:108BB000BDF808202AB12088154905EB004003F0D4
:108BC0003FF907B03046F0BDC42D00200804030073
:108BD00054686520726571756573746564205458B6
:108BE0002F5258207061636B6574206C656E6774DA
:108BF0006820697320746F6F206C6F6E67206279D4
:108C00002025752F2575206F63746574732E000001
:108C10005404030030B5044685B000211B4804F01D
:108C2000E8FF00282FD00025204600F030FF68B173
:108C3000112812D086281BD0A0F54051023903D04C
:108C40000146204605F04CFE294607E005B02946BE
:108C50002046BDE8304001F02BBD0121204601F047
:108C600027FD05B00021BDE83040084804F0F5BFFD
:108C7000142207496846FDF7F9FBADF80240684643
:108C800000F098F9E0E705B030BD0000D52B0020DA
:108C900068FF02007FB50C4610B1012004B070BD22
:108CA0002079002638B141F61D5501281BD0022835
:108CB00026D00F20F2E70220207102960396E0688A
:108CC0000190694601A805F03FFB50B102988188E8
:108CD000E18000882081BDF80010029805F0B2FB09
:108CE000DCE70A20DAE70A4B6A460021A01D05F0FE
:108CF000E7FA38B1064918398E61CE610A28CDD11C
:108D00002846CBE702488188019805F09BFBF5E7F0
:108D1000F82C00202DE9F0470025DFF88C803CE09E
:108D20006068002100EBC506012032789146FDF70E
:108D30008AFBD4E9062300EA020701EA030C57EA9A
:108D40000C0728D082438B434846C4E9062303F02E
:108D5000BBFD32788246914601200021FDF773FB6E
:108D6000D4E9042300EA020401EA03074A46504614
:108D70000021FDF768FB44404F403C430BD1707825
:108D8000012801D0012100E00021726881EA0A0176
:108D90000AB1484690476D1CEDB298F80000444671
:108DA0008542BDD3BDE8F087982C002010B5002186
:108DB000024801F099FF80F3100010BD343C002000
:108DC0000E4910B50A784C780023A24212D0521CEA
:108DD000D2B20A70022A00D10B70084A0B780C320A
:108DE00052F8232002608868104420F07F40886099
:108DF000012010BD0360002010BD0000B82C002031
:108E000013460A460021FFF785BE00002DE9F8430E
:108E1000104D0F4680461E4691466946286801F06F
:108E2000BEFE040014D01C21FDF747FB0120207179
:108E3000C4F81490380BC4F80080C4E90260694695
:108E4000286801F0CDFE05F0CFF90020BDE8F883D9
:108E50000420FBE72001030010B503780022072B54
:108E600006D2DFE803F005040610202930000A705E
:108E700010BD01230B7003898B818388CB81C0686F
:108E800088600A7410BD02220A7002898A81828871
:108E9000CA81C2688A60807D062802D000200874DA
:108EA00010BD0120FBE703220A70C2888A81028973
:108EB000CA81C068886010BD04230B70C088888197
:108EC000CA818A6010BD0520087010BD70B5064DBE
:108ED0000646002455F8241009B130468847641C22
:108EE000042CF7D370BD00009835002030B504463F
:108EF000006887B00D46806800281FD0182168469A
:108F0000FDF7DBFA0195A0680590207910B10128E2
:108F100010D107E001208DF8000020690290E06880
:108F2000039005E002208DF80000E0680003029045
:108F300060690490206881686846884707B030BD42
:108F400070B586B015460C00064619D0112C17D006
:108F5000082C15D014216846FDF7AFFAADF8026071
:108F6000304601F065F8ADF804000D2C0AD0862CCF
:108F70001CD007208DF800000294684600F04CF8E1
:108F800006B070BD03208DF8000025B12878C00719
:108F900001D0012000E002208DF8080000208DF8AB
:108FA0000C0041F20110ADF80A00E6E706208DF84A
:108FB0000000E2E710B50446408801F039F8A080CF
:108FC000024801682046BDE810400847DC2B00201D
:108FD0002DE9F04107460024064E074D05E000BF8D
:108FE00056F8241038468847641CE8788442F7DB3A
:108FF000BDE8F08138330020FC2B002010B504467A
:10900000408801F015F8A080024801682046BDE8BC
:109010001040084714000300014909680847000090
:10902000680003007047000070B586B00446142144
:109030006846FDF742FAA0890125A0F54040ADF849
:10904000040020782A4E062833D2DFE800F03203ED
:1090500003032C48A08900F0BDF930B9E08943F63C
:10906000FE71A0F54040884223D8A07B8DF808000F
:10907000207803280FD000208DF80900A068039005
:10908000606850B109208DF800006068049068465F
:1090900004F00AFA0DE00120EEE708208DF8000048
:1090A0008DF81050F3E7A08900F094F908B1E08939
:1090B00030B17078002801D004F026FB06B070BDF6
:1090C000606820B10B208DF800007570DFE70A2082
:1090D0008DF80000BDF8040004F0A0FBF5E71320B4
:1090E0008DF800004FF6FF70ADF80400CFE70000E8
:1090F000EC2B002038B504460E480078A8B1A4F542
:109100007F40FF380FD0684604F0A0FF78B10521FA
:10911000017001210171C480684604F0A5FF05F0CB
:1091200055F8002038BD042038BD022038BD082085
:1091300038BD0000002D00200C4808B5007888B12B
:10914000684604F083FF78B106210170684604F098
:109150008BFF0748017809B10121017305F036F84A
:10916000002008BD022008BD082008BD002D0020F9
:109170005C360020F0B587B014216846FDF79DF9F4
:109180002B4C207818B16846FFF7A0FE4EE0201D5A
:1091900001F08CFDB8BB4FF010204169000402695A
:1091A00040694B1C01D100FB02F122480022016101
:1091B000A1F54051C160204902F04CF9002820D1AE
:1091C0001F481C238C221D49006801F0D5FC03F0C8
:1091D0005BFF051E14D0022812D000270126062DA1
:1091E00012D005A804F032FF88B106700C2D18D2F9
:1091F000DFE805F0170F170F1716171617111311C1
:109200000B2007B0F0BD11E026706760BBE70820B7
:10921000F7E7077105E0032100E00221017100E09A
:10922000067105A804F020FF04F0D0FF0020E8E755
:10923000002D0020B02D002030010300A8350020B3
:109240009800030038B5040014D0694605F07CF896
:10925000A0B1BDF8000000EB8001094800EB8100DF
:10926000C16849B1A17A39B1C168491EC160002005
:10927000A07238BD052038BD062038BD0A2038BD93
:10928000343600201FB501A9684605F019F804B06E
:1092900010BD07B513460A466946002005F010F8D0
:1092A0000EBD07B513460A460021684605F008F8CA
:1092B0000EBD20B119B1006808600020704705207C
:1092C00070470000F8B50D46040018D0BDB16946DE
:1092D00005F03AF8A8B1BDF800000B4900EB80009A
:1092E00001EB800001210C30666801F0E2FC2E6089
:1092F00060680C3068600120A0720020F8BD052075
:10930000F8BD0A20F8BD00003436002018B1032350
:10931000002206F0D5BC052070470223002206F08B
:10932000CFBC12B1022306F0CBBC05207047000071
:10933000084910B50A69042A0AD0074A096942F89F
:10934000210004480121103001F0B3FC002010BDC1
:109350000C2010BDE02C00209835002038B50446C4
:1093600009480D46007858B164B16946284606F0B0
:10937000A1FD002803D1BDF800102180658038BD13
:10938000022038BD052038BD002D002010B5044650
:109390000E48007898B1A4B12188022913D80C4A4C
:1093A00001EB810002EB800260885289C31C93426A
:1093B00009D806F073FD00202080608010BD0220D7
:1093C00010BD052010BD042010BD0000002D0020A0
:1093D0003436002043F6FE71A0F54040884201D8A3
:1093E000012070470020704710B504460078182807
:1093F00002D1FEF721FB207010BD10B504460078A5
:10940000182802D1FEF718FB207010BD70B50D466C
:109410000446B0F89810D0F894000122FDF7B6FF8A
:1094200000B1057004F13C0204F1940104F1540010
:1094300072DF70BD70B513460022064615468629B8
:1094400002D0112902D002E0012200E001250D4CDA
:1094500073B1A179FEF714FB2A4661793046FEF715
:109460000FFB0022A1783046FEF70AFB002203E042
:10947000A178FEF705FB2A4661783046BDE87040CA
:10948000FEF7FEBA142C0020F7B517460E0011D0D7
:109490000098002560B100242146684601F0EBFBEE
:1094A00018B1A0B23946B0476D1C641C142CF3D31C
:1094B0002846FEBD0020FEBD406804F0E7BD000068
:1094C0000EB517A19DF8080020F00F00401C20F0F9
:1094D000F00010308DF808000A2202A87CDF08B1E5
:1094E000FDF7DEFB40F2413078DF08B1FDF7D8FB35
:1094F0000020009001904FF4A071ADF80400ADF889
:1095000000104FF4C8704FF40271ADF80600ADF8CA
:10951000021068467ADF002801D0FDF7C1FB0EBDBE
:109520004E6F726469635F48524D000010B5088841
:109530000C46A0F52061773909D108480321A3889A
:109540000088628801EB004005A102F080FC214602
:10955000BDE810400E48FEF7B2BD0000F82D002017
:109560004741545420415454204D5455206F6E208F
:10957000636F6E6E656374696F6E20307825782036
:109580006368616E67656420746F2025642E000037
:10959000882E002070B508B1012070BD194C00253F
:1095A000207B08B1257301E000F0A0F8207808289E
:1095B00026D2DFE800F02504080C10251420BDE8B1
:1095C000704000F021B8BDE8704000F07DB8BDE803
:1095D000704000F05FB8BDE8704000F03BB86088B4
:1095E000084900EB8000283901EB80004068BDE8A5
:1095F000704003F029BD6560BDE8704003F032BDE6
:109600000F2070BD5C3600201149F0B48A1C002088
:109610000346A1F128050C18A67A4EB1A37200EBFF
:10962000800405EB8404E66816B9247C012C0AD07A
:10963000401C80B20228EED30B704B804B60F0BC14
:1096400041F61D5070471080F0BC00F03DB800009E
:109650005C3600200C48418801EB8102A0F1280112
:1096600001EB8201CA6852B105210170074802214D
:109670008180016800230122054801F055BE0422C3
:1096800002704968F6E700005C360020082D0020D3
:10969000B02D002038B50A49084803240B684268F9
:1096A000898803EB810153880470DB1C00201B04B4
:1096B00000909B0B034801F0A7FF38BD5C360020EB
:1096C000082D0020B02D0020074910B54888091D3D
:1096D00004F08AFE18B1BDE81040FFF7DBBFBDE81B
:1096E0001040FFF7B7BF00005C360020F0B51F4800
:1096F0001F490125067802248B88A0F12802082E34
:1097000019D2DFE806F00418181B222F2F17018941
:10971000491C01810021418080F80C1001EB81037C
:1097200012F8233043B100234418491C89B2A372B4
:109730000229F3D30570F0BD0123F5E74268528892
:10974000D21C1A448A800470F0BD46880D6806EB6E
:10975000860602EB860256680E60556013818C8087
:10976000062100E007210170F0BD00005C360020FA
:10977000082D002030B501888488224D85B05029FD
:1097800024D0522902D0542931D103E0204600F0E0
:109790005BFF2CE014221C496846FCF767FEADF81D
:1097A0000240204600F044FCADF8040000F022F92D
:1097B000002269792046FEF763F9002229792046C4
:1097C000FEF75EF96846FFF7F5FB10E0017B012923
:1097D0000DD1817A01290AD10089A0F524510239DD
:1097E00005D10121204600F063FF06F08FF800222A
:1097F0000649E878FEF7E6F805B0BDE8304005F028
:1098000027B90000D42B002090FF0200996F0200BE
:1098100010B50446007800280FD1608800F014FFCE
:10982000608800F081F9002807D00449608801228F
:109830000979BDE81040FEF723B910BDD42B0020F4
:1098400010B5124C00202070FEF7F6F8A070FEF75D
:10985000F3F8E070FEF7F0F82071FEF7EDF86071B4
:10986000A17818290FD0E17818290CD0217918296E
:1098700009D0182807D00121601C04F0B3F9012099
:109880002070002010BD032010BD0000D42B00204C
:109890007CB50446007808282FD1607A38BB207A3E
:1098A0004FF6FF7501280DD0072802D0082824D1D3
:1098B0001EE0A08800F0FAFAA8421ED0012100F0B4
:1098C000F7FE1AE0A0886A46012103F005FD70B991
:1098D0000198007858B1A08800F0E8FAA8420CD0AE
:1098E000084901220979FEF7CBF805F0B1F804E048
:1098F00004480021401C04F0B0F9BDE87C4006F0AB
:1099000005B80000D42B002010B504460A48417861
:109910002046FEF79DF868B10848002101EB41029E
:1099200000EB82025288A24201D1C8B210BD491C8C
:109930001429F3D3FF2010BDE62B0020283100208E
:1099400070B5094D094E002404EB440005EB80007E
:1099500071784088FEF77CF820B1641C142CF3D396
:10996000FF2070BDE0B270BD28310020E62B002042
:109970002DE9F0418046024601200021FCF763FDFD
:109980001A4F05460E467868FDF716FA00280CD1E6
:10999000174CD4E9062110462A4001EA06031A436F
:1099A00005D0A843B143C4E90601BDE8F0814046B3
:1099B00002F08AFF30B1D4E9040128433143C4E9FD
:1099C000040105E0D4E90410A943B043C4E904103C
:1099D000D4E9060128433143C4E90601A168786847
:1099E000BDE8F0410022FDF7A3B900007C000300B0
:1099F000982C00201CB5054AD2E90212CDE90012CC
:109A00000022694603F08DFC1CBD0000A8FF020087
:109A100003484FF6FF7181800121017000207047DB
:109A2000E02B00202DE9FC41804600F001FB0024E2
:109A300003250127A0F57F412646FF3908D06A4655
:109A4000082103F049FC18B90198841D868805682F
:109A500032462B4621464046B1DF042804D0082870
:109A600004D00B2808D002E0112000E00020002FD5
:109A700000D10B20BDE8FC810027A80701D50125F6
:109A8000E6E73443F5D0002426460325E0E72DE938
:109A9000FC41804600F0CCFA0646A0F57F40FF3836
:109AA0000ED001252A466D1C0027ADB26B46082159
:109AB000304603F03BFC040006D0072C25D025E0FF
:109AC00043F20200BDE8FC81019903230A1D0B60EB
:109AD0004046891DB2DF040004D00C2C09D0052CAF
:109AE00009D009E032460821104603F095FC0446EF
:109AF0000CE0012700E000240821304603F078FC48
:109B000000B10324002FCDD100E00C242046D9E77A
:109B100004488088A0F57F41FF3901D004F0A2BF3E
:109B200070470000E02B00200EB502A9019100F063
:109B30007FFA6A46012103F0CFFB08B100200EBD79
:109B4000019800780EBD00002DE9F04107464FF660
:109B5000FF760A48B3DF10B10320BDE8F081074C5F
:109B600043F20305A41E324661883846AFDFA8429F
:109B7000F3D16088401C6080F5E70000E22B0020F4
:109B8000428800EB82020C328A4201D902207047DF
:109B90008188A1F57F42FF3A03D0008808B10020F8
:109BA000704701207047884204D20068401C01D0F1
:109BB000012070470020704710B51249124804F088
:109BC0001AFF114C81B2103C6068401C60600F4865
:109BD000FEF7F0F958B1082809D0132807D011284A
:109BE00005D043F20141884201D0FDF759F8606881
:109BF0000321B0FBF1F201FB120000B10120207043
:109C000010BD0000D42F0020982B0020882E0020AB
:109C100070B5CCB00024054644949DF810010E4662
:109C200020F00F00401C20F0F00010308DF81001E3
:109C3000087B8DF811019DF812011C2120F006000F
:109C4000801C8DF812013DA8FCF737FC9DF8F4004C
:109C50003E9440F010008DF8F40044A84094CDE903
:109C6000414001208DF82E0142F637204394ADF893
:109C70002C014A94707B8DF82801B07B8DF8290166
:109C80009DF82A01142120F00600801C20F0180005
:109C900040F001008DF82A0145A8FCF70EFC4BA806
:109CA00045904AA846906A460021284600F012F8DE
:109CB000ADF81C01F420ADF81E41ADF82001CDF83F
:109CC00024D1E88805F1080345AA3DA9AADF4CB0D4
:109CD00070BD00002DE9F041044640799046002512
:109CE00000B1042594F8220008B145F00205CAB27B
:109CF000FF2908D9090A88F8012045F0010588F8EC
:109D00000210032602E088F801200226B4F84C0075
:109D100008B145F0100500271BE000BF94F84E1075
:109D2000B21C91420BD2B4F84C0004EB4701C01BAB
:109D3000420004F124002431FCF798FB0DE004EB11
:109D4000470008EB0601808C0870000A4870D6B204
:109D50007F1CB4F84C00B842E0DC34F84C0FC01B58
:109D6000208088F800503046BDE8F0813EB502788A
:109D700002230C46B3EB520F17D1B0F80110ADF827
:109D80000010C1788DF802108188ADF80410807938
:109D90008DF8060002AA01A92046FCF7C3FE0322A3
:109DA00002A96846FCF79BFB08B100203EBD0120DC
:109DB0003EBD000010B50C46FFF7A6FDFF280CD0F5
:109DC000074900EB400001EB8000416821600189F8
:109DD000A180807AA071002010BD052010BD000078
:109DE0002831002070B5018890B0102959D1011D8B
:109DF0002C226846FCF73AFB9DF804004FF6FF76EC
:109E0000032134466D46B1EB500F2AD003F0BAFB64
:109E10009DF8040040080ED001280CD0022820D163
:109E200018E00D99281D1131FCF718FE18B100BF7C
:109E3000BDF82C4015E00CAA0BA9072003F076FB17
:109E40000028EED10DE00D99281D491CFFF78EFF6B
:109E50000028EDD10CAA0BA9072003F067FB00280E
:109E6000F1D1BDF80000291D00F030FEB44218D039
:109E7000BDF80000214600F0C5F8BDF80000ADF8BF
:109E80002E000020ADF83040074E8DF82C000BADB1
:109E9000044600BF56F8241028468847641C022C4C
:109EA000F8D310B070BD0000BCFF0200094A0021C9
:109EB00001EB410332F82330834205D101EB41002D
:109EC00002EB800040887047491C1429F0D34FF6FC
:109ED000FF707047283100203EB50C46054603F060
:109EE00051FB0BE0BDF80000A04207D028460299C4
:109EF00000F02EF810B1BDF800003EBD01AA694681
:109F0000072003F013FB0028ECD14FF6FF703EBD95
:109F100010B50D4C18200D4A607000204FF6FF71EF
:109F200000EB400302EB8303401C59801428F7D355
:109F3000FDF782FD6070182803D0012020700020FA
:109F400010BD032010BD0000E62B002028310020AA
:109F50002DE9F0410C46054600F1110701F111060B
:109F60001022491C401CFCF7BAFA48B9681C00F0E2
:109F7000F9F928B1601C00F0F5F908B1012400E0FE
:109F8000002431463846FCF769FD3B780222B2EBEB
:109F9000530F0CD00321B1EB530F08D03378B2EB41
:109FA000530F04D0B1EB530F01D0012100E0002189
:109FB000084201D18C4302D00120BDE8F08100208D
:109FC000FBE7018811B9421892780AB10120704765
:109FD000491C0829F7D30020704710B50C460346EA
:109FE000FFF7EFFF00280AD018882188884205D1A2
:109FF0000822A11C981CFCF772FA08B1002010BDC1
:10A00000012010BD03F05EBC70B50446FFF74EFFA3
:10A010000546204603F063F94FF6FF7104468D4272
:10A0200003D014B9284603F04DFC204670BD000053
:10A0300010B5FFF769FCFF2805D0044900EB40008C
:10A0400031F8200010BD4FF6FF7010BD2831002000
:10A050003EB5044603F096FA0EE0019920464631DB
:10A06000FFF7BBFF28B9019920462A31FFF7B5FF5A
:10A0700010B1BDF808003EBD6A4602A9072003F0F2
:10A0800055FA0028E9D14FF6FF703EBD10B50A49D8
:10A0900041600A4800F00AFE58B902F087FA074901
:10A0A0001C238C22087404488C39001F006800F0BF
:10A0B00063FD002010BD000024010300F8360020DD
:10A0C0002DE9F0412D4F002518B17D600120BDE83C
:10A0D000F0810879012258B1294E01280CD0274C73
:10A0E0004FF002080834022821D0032842D128E08A
:10A0F0000A7102F0B7FF3BE05FF0000000EB800167
:10A1000016F82110022908D0401C80B20228F5D38D
:10A110003A707D6041F61D50D9E700EB800006F8EB
:10A12000205006EB8000406802F08EFF20E00D71A9
:10A13000A4F80480002301221248216801F0F4F8F9
:10A1400016E00D71206802F07FFF0D492368283169
:10A15000498801EB810206EB8201D1F804C0C4F802
:10A1600000C04B60A3880B81A4F8048006F822503D
:10A170000028ACD07D600E20A9E70000002D002053
:10A1800034360020B02D00200146034802888A4260
:10A1900000D0002070470000803000202DE9FC5FD7
:10A1A0000E008346DDE90C47C6F100009846924652
:10A1B000814600D40846012503E000BF90FBFAF079
:10A1C0006D1C5045FADAA84500D9454624B1002E49
:10A1D00001DB780700D5641EB80702D5B8F1000F7F
:10A1E0000AD0F80708D13CB1A54205D22021584633
:10A1F000641EFEF7C9FAF6E7002E02DA4E462D215C
:10A2000002E0780703D52B215846FEF7BDFA07F088
:10A21000030002280BD1B8F1000F08D13CB1A542D0
:10A2200005D230215846641EFEF7AEFAF6E7CDE9B6
:10A230000047434652463146584605F00DFBBDE8FF
:10A24000FC9F000070B50D46044600684FF488710D
:10A2500002F042FA4FF49071206802F03DFA4FF498
:10A260009271206802F038FA4FF4A271206802F06F
:10A2700033FA20681249C0F8041320686907000BFC
:10A2800040B2090E002806DA00F00F0000F1E020CD
:10A2900080F8141D03E000F1E02080F8001420682D
:10A2A0000121000B40B200F01F02914040098000E4
:10A2B00000F1E020C0F88012C0F8001170BD00006D
:10A2C00010030200024600201268930702D05307D1
:10A2D00002D47047500714D502F00300012802D0C1
:10A2E00002280CD105E0C2F383100B68801C1844CF
:10A2F00004E00223086803EB925210440860012036
:10A300007047086800EB9253C2F38910401CEEE7D7
:10A310000248007A002800D001207047F83600205B
:10A32000F0B58488A518944200D82246A41AC288A1
:10A33000D6189A4200D81346D21A4B880788BB42D7
:10A340000CD34088834209D88888A04206D3A8420B
:10A3500004D8C888904201D3B04201D90020F0BD92
:10A360000120F0BD0021425C0AB101207047491C68
:10A370001029F8D300207047800701D000207047D3
:10A38000012070470A4810B5807860B1002401E0D0
:10A39000022C06D02046FDF76FFF641C042CF7D377
:10A3A00010BD0324F6E7BDE81040FDF789BF0000AB
:10A3B000B42B002003480179C90702D00078FEF7CA
:10A3C000BBB87047B42B0020F721018017214180D2
:10A3D000002101714171FB2181711B21C171704705
:10A3E0002DE9FE4F2B4D984691460F00824601D035
:10A3F00000260DE0684600F095FB6A4600215046B5
:10A4000002F0D9FE2878009E10B99DF8090098B195
:10A410004A463146504604F0EFFD0446014600220C
:10A420005046FFF707F80D2C32D008DC84B3082C17
:10A430002ED00B2C0BD12BE00520BDE8FE8F112C6C
:10A4400010D0862C1AD0A4F54050023820D0032515
:10A45000B8F1000F04D0324621465046FEF770FD99
:10A460002846EAE73A4629795046FDF709FB4A466D
:10A47000E9785046FDF704FB0025E9E73A462979DB
:10A480005046FDF7FDFA4A46E9785046FDF7F8FADE
:10A490002546DDE7142C00202DE9F041204F0E4623
:10A4A000154604463978FDF7D3FA002835D0204602
:10A4B00002F078FE50B32046FFF7BAFD80462046F2
:10A4C000B978FDF7C5FA08B1012700E00227204658
:10A4D00003F010F90028404602D0FFF795FD0DE08B
:10A4E000A8F57F41FF3909D0072102F081FF010063
:10A4F00004D0052902D0204604F006FA2B46324645
:10A5000039462046BDE8F041FEF704BB2A463146F5
:10A510002046BDE8F041FEF773BCBDE8F0810000C5
:10A520000C2C002070B5094D0646E978FDF790FA2D
:10A53000044629793046FDF78BFA0146224630461B
:10A54000BDE870400123FFF74BBF0000142C002032
:10A550002DE9F047394E002780463D46DFF8E09070
:10A56000D6F804A057E003D00446D0F81C8035E0AC
:10A5700099F8002002EB4201521CD2B289F8002067
:10A5800009EBC10199F80230091D9A4201D189F8FD
:10A59000005048680A780446012A12D0022A02D0E4
:10A5A000032A3BD108E004F0F1FE00B10127257435
:10A5B00034E00574C06900E070680028F9D170606B
:10A5C0002CE0207C50BB88686060C868A060086987
:10A5D000E0604869A061F07800B165606268B168C8
:10A5E000184B501A20F07F40984202D2A1680844CC
:10A5F00006E0881AA16820F07F40814202D9081A3B
:10A60000206000E0256065600120A5602074204680
:10A61000E56104F09DFEB8F10000A4D199F80010A6
:10A6200099F801008142A3D117B97168514502D050
:10A630000120BDE8F0870020FBE70000B82C0020D7
:10A6400074340020FFFF7F0030B585B0054600243C
:10A6500014216846FBF731FFA5F57F40ADF80250A5
:10A66000FF3815D02846FFF7DDF998B10B2815D033
:10A67000112811D0A0F54051023903D001462846D7
:10A6800004F02EF909482246C1782846FDF7F8F96A
:10A6900005B030BD0E2002E00124F3E70F208DF855
:10A6A00000006846FEF786FCECE70000D42B002093
:10A6B0000A4602498978FDF7E3B90000D42B00204F
:10A6C000F8B5054600780C46002620420FD1002040
:10A6D0008DF800006846FCF77FFB2878204202D105
:10A6E0002043287001269DF80000FCF799FB3046B6
:10A6F000F8BD00002DE9FF410026234800F0D3FA01
:10A700002148001F074600F0CEFA204C60680090F8
:10A71000A56800E000986946284004EB80000C30F2
:10A72000FFF7D0FD0028F5D101AA009901EA050341
:10A7300004EB8303491CDB6842F82030401C009185
:10A740000228F2D3019800F0030001280BD0022860
:10A7500010D10198032101EB90500099BDF80A60D7
:10A7600001EB900005E00198BDF80A60C0F383108A
:10A7700008440090384600F093FA08B100986060F1
:10A7800004B03046BDE8F081303C0020183800208D
:10A79000ACB04FF40041002001F0C0FB08B1FCF761
:10A7A0007FFA01F02BFA04F07FFE4D490320FDF7FC
:10A7B00079FE08B1FCF774FA69460020FDF7A4FDA4
:10A7C00008B1FCF76DFA9DF80000022874D000264D
:10A7D00001F0C2FC08B1FCF763FA01F09BFE08B17E
:10A7E000FCF75EFA002469460120009401F0F6FCB3
:10A7F00008B1FCF755FA684601F09CFD08B1FCF77A
:10A800004FFAFEF75DFE3749374800F0E2FA08B12B
:10A81000FCF746FAAC216846FBF74FFE02208DF8A4
:10A82000000001208DF80200062103258DF87C0030
:10A830008DF80310ADF810504FF496702B4922900C
:10A84000059144F250602390294829902648694692
:10A850002030FCF7CAFD08B1FCF722FA224801219A
:10A860002030FCF7BFFD04F0A9F904F06DF81C21BD
:10A870006846FBF722FE4FF42030CDE900404FF44C
:10A880007020029018488DF80C5064388089ADF81B
:10A890000E0018480590184806908DF8104068463C
:10A8A000FDF746F808B1FCF7FBF903F019F8134877
:10A8B000008805EB004000E00FE011A101F0BCFAB8
:10A8C000FCF7C8FA3046FCF709F900BF01F0A4F91B
:10A8D0000028FBD101F054FCF8E7012678E70000DE
:10A8E000FD8302002D950200EC2E0020A82B0020F5
:10A8F000F1CD02003DCE0200C78A0200F82D0020F3
:10A90000486561727420526174652053656E736F7F
:10A9100072206578616D706C652073746172746506
:10A92000642E000070B5144682880E4605462088C5
:10A93000111D0144921C994201D8FE2A01D90C2014
:10A9400070BD521C32542088FF21401C80B22080F0
:10A9500031542088401C80B220808119288804F05E
:10A9600065FF2188084480B22080AA8842B1A96886
:10A9700041B13044FBF77AFD2088A9880844208043
:10A98000002070BD072070BD2DE9F047C788044640
:10A99000181D16468946B0FBF7F1B0FBF7F207FB2E
:10A9A00012009A193A44D21CB2FBF7F2DDF820A04B
:10A9B00001E02468491E0029FBD13D1A8846B542B2
:10A9C00016D818E0BAF1000F05D0211809EB0800DD
:10A9D0002A46091D04E0204409EB08012A46001D0F
:10A9E000FBF744FD00202468761BA844B74201D938
:10A9F000354600E03D46002EE4D1BDE8F08700007A
:10AA000030B5024659B101F0B5FA0021074C09E012
:10AA100004EB810315685B88AB4202D11160002012
:10AA200030BD491C8142F3D3052030BDC42D002028
:10AA3000F8B50F46017814460546012901D168781A
:10AA400030B12088821C9A422DD8012902D006E01C
:10AA50000720F8BD69780144891C994223D8181A47
:10AA6000801E86B2ADF800602188B81C0844694693
:10AA70007DDF0028EDD12878022805D1BDF800102F
:10AA8000B14201D809210AE00821012805D16878DE
:10AA9000B04202D8ADF8000001E0ADF80060BDF8AA
:10AAA0000000FE2801D90C20F8BD2288401CB854B3
:10AAB0002088401C80B2208039542088401C20808F
:10AAC000BDF80010084420800020F8BD70B5054690
:10AAD0000C004FF0FF0020D04FF6FF76B5421CD09F
:10AAE0000E48012241782846FCF7CAFF2846FEF7A7
:10AAF0000BFFFF2803D1FEF723FFFF280DD0084BE3
:10AB000000EB400203EB82014D8023F822602268B3
:10AB10004A60A2880A81A2798A7270BDE62B002061
:10AB200028310020034A00219268C0E90021816099
:10AB300070470000142C002070B54FF6FF750E46CC
:10AB4000A84201D1002000E0401C84B208E0214668
:10AB5000304603F076F808B1204670BD641CA4B2FC
:10AB6000FF2CF4D9284670BD10B5FBF79EFB08B149
:10AB7000002010BD112010BD10B531B1B2FBF3F4AF
:10AB800003FB14241CB1092010BD0E2010BD016070
:10AB90000021416081608281C381084610BD70B58B
:10ABA0000C460546FBF736FB002802D021882868B2
:10ABB000084470BD10B50A8849888A4203D1FBF762
:10ABC0006BFB012010BD002010BD70B50C46054682
:10ABD000FBF745FB002802D061882868084470BD57
:10ABE00010B50A8849888A4203D1FBF72FFB012060
:10ABF00010BD002010BD01F01F0301229A40D24376
:10AC0000490900EB8100114600F059B80A4601F0ED
:10AC10001F030121994010B552090C4600EB820038
:10AC200000F05DF8204000D0012010BD2DE9F0417A
:10AC300080460D460024481E012101EB501716E006
:10AC400058F82400C04390FAA0F0B0FA80F0202811
:10AC50000CD200EB4416AE4208D231464046FFF714
:10AC6000D5FF0028ECD13046BDE8F081641CA74236
:10AC7000E6D82846F8E74A0950F8220001F01F02FA
:10AC800001219140084000D00120704701F01F03CE
:10AC900001229A40490900EB8100114600F029B8D1
:10ACA000002100F017B8012100F023B8012100F0C5
:10ACB00016B808B56A46FBF744FB009808BD08B50E
:10ACC0006A46FBF724FB009808BD08B56A46FBF707
:10ACD00038FB08BD08B56A46FBF719FB08BD08B587
:10ACE0006A46FBF707FB08BD08B56A46FBF7F6FAAC
:10ACF00008BD08B56A46FBF7FDFA009808BD08B51F
:10AD00006A46FBF72BFB009808BD38B504460025C2
:10AD10008DF800506846FCF75FF8216862680868A3
:10AD200090420ED9401E08600178A38AE26801FBB8
:10AD30000325227A2168101AC0B20A79824200D211
:10AD400008719DF80000FCF76BF8284638BD38B54F
:10AD5000054600208DF800000C466846FCF73CF8DC
:10AD6000E868A98A201AB0FBF1F12A681068431C30
:10AD7000136001709DF80000FCF752F838BD10B563
:10AD800030B1017A42680368891AC9B21A6006E0D4
:10AD90000E2010BD03681A68541C1C601170491EF7
:10ADA000C9B2F7D2006800210171084610BDC2087F
:10ADB00000F007030120895C98400840704710B5F7
:10ADC000C20800F00703885C01249C40204388549B
:10ADD00010BD10B560B10161F72120F8021B20F809
:10ADE000021BFB2100F8021BFFF7EEFA002010BD4A
:10ADF0000E2010BDF0B5858893B00C46002D39D1DA
:10AE0000018800263E4F24293BD006DC102909D0BA
:10AE100011290CD0232958D14FE03A290BD05529BC
:10AE200053D129E00146204602F016F84DE0A01D5E
:10AE3000FFF7CAFA49E02246408934F8061F8142EA
:10AE400000D808466080172800D21720608010695B
:10AE500070B1607960B1D7E90001CDE90301ADF8C7
:10AE60000E506088ADF81000136903A9104698478A
:10AE70006671267113B0F0BD0146204602F03CF821
:10AE800023E0011D2C2206A8FBF7F0FABDF81800FC
:10AE9000BDF81C2004EBC0014A732269AAB1D7E9AE
:10AEA0000423CDE90423ADF81200487B8DF814008B
:10AEB0002269204604A9904707E0017A207B884256
:10AEC00000D201462846FDF747FEA07A0028D1D0DF
:10AED000E1882846A5DF012570B11128CAD001F00C
:10AEE000DBFB0246074808A1008813B005EB0040D1
:10AEF000BDE8F04000F0A4BFA672E572BAE700001A
:10AF0000C4FF0200C42D002073645F626C655F673C
:10AF1000617474635F65786368616E67655F6D74A3
:10AF2000755F726571756573742829207265747513
:10AF3000726E65642025732E0000000020B1027837
:10AF4000DE2A03D0082070470E2070474180002081
:10AF5000704760B159B10278DE2A0AD009684160B1
:10AF6000DE2101704FF6FF714180002070470E20F6
:10AF70007047082070477FB5054600294DD0002D49
:10AF80004BD008780C46DE2847D1A88861888842D3
:10AF900002D1204604F00AFD2888012825D0022885
:10AFA0003BD011283AD0512837D135F8040F6188A9
:10AFB000884232D1A978A81C02292ED1017A04290D
:10AFC00003D0062901D0052927D1002100910222B2
:10AFD0008DF8002001914FF4C07202910391ADF8F9
:10AFE0000420007A05280FD010E0297A2046012994
:10AFF00013D1A988428891420FD10121017204B076
:10B00000BDE8704004F0D2BCADF804102888694651
:10B01000B0DF002801D0616888477FBDA8886188BB
:10B020008842FAD14FF6FF7060807FBD00F180400A
:10B030000068002800D00120704708B500F180406A
:10B04000002101600068009008BD000070B50B4C45
:10B05000207808B185250FE00020A06060602061A5
:10B06000E060074801F054FB054601F09FFA08B97B
:10B0700001F038FB01202070284670BD8433002089
:10B080003989020038B500258DF800506846FBF775
:10B09000A3FE074CE068401EE060E06810B901F0D4
:10B0A00047FBA5709DF80000FBF7BAFE38BD000015
:10B0B00084330020F0B505460478154889B016465B
:10B0C00040F82420124A08690832A2F10C0742F81D
:10B0D0002400487F385520226846FBF7C7F90494BE
:10B0E0002878385C48B10EB10A4A00E0002269466F
:10B0F000281D01F099FD09B0F0BD0EB1064A00E02F
:10B100000022694605F10C0001F060FCF3E7000045
:10B11000782C002009F7020055F502000FB408B59D
:10B120000399002904D004AA00926A4600F00FF89F
:10B1300001B05DF814FB10B582680446002A05D002
:10B14000D4E90403216898470020A06010BD2DE9D0
:10B15000FC4791460C00804676D014F8011B39B1AB
:10B1600025290ED04046FDF70FFB20780028F4D1AA
:10B1700098F80C00002867D04046BDE8FC47FFF770
:10B18000DABF0020012221782B291BD02D2902D0E3
:10B19000302908D102E040F0010001E040F0020057
:10B1A000641C002AEFD100252A290ED02178A1F1B4
:10B1B00030020A2A11D205EB850201EB4205641C1C
:10B1C000303DF1E740F00400EAE7D9F800100B1D2C
:10B1D000C9F800300968641C0D44217800232E2929
:10B1E0000BD114F8011FA1F130020A2A05D203EB9A
:10B1F000830201EB4203303BF3E76C290DD0682951
:10B200000BD0692921D00BDC252918D0582931D041
:10B2100063290ED0642915D117E014F8011FECE75B
:10B22000702969D0732932D075291BD0782909D1AA
:10B2300020E0D9F80000011DC9F80010017840464F
:10B24000FDF7A2FA641C90E76CE0D9F800100A1D23
:10B25000C9F800200968CDE900500A224046FEF7EF
:10B260009DFFEFE7D9F800100A1DC9F80020096812
:10B270000A2206E0D9F800100A1DC9F80020096862
:10B280001022CDE90050404604F0E6FADAE7D9F89A
:10B29000001000270A1DC9F800200E68C00705D15C
:10B2A00012E04046761C7F1CFDF76EFA31780029CB
:10B2B000F7D104E0202140466D1EFDF765FABD423E
:10B2C000C0D9002DF6D1BDE74EB13046FBF700F9ED
:10B2D000074604E0202140466D1EFDF755FABD42A9
:10B2E00006D9002DF6D103E04046761CFDF74CFA56
:10B2F00031780029F8D1A5E7D9F80000011DC9F877
:10B300000010056830214046FDF73EFA782140469E
:10B31000FDF73AFA08200021CDE90001034610228A
:10B320002946B0E7BDE8FC872DE9F84F2B4E040015
:10B330009A4630884FF001031546894603EB0040DA
:10B3400024D0216800292BD0002D32D062684946D4
:10B350004FF010071268A2F1010C1CEA090F11D17D
:10B3600098466A432046FBF792FB00282AD02068C3
:10B3700053462A46066901B049462046B446BDE810
:10B38000F04F6047164B17A2009721E00E21009165
:10B39000134B1EA21FA100F062FD0E20BDE8F88F26
:10B3A000082100910E4B26A21AA100F058FD08209A
:10B3B000F4E7092100910A4B24A216A100F04FFDE9
:10B3C0000920EBE700973188054B214A08EB014043
:10B3D00010A100F044FD1020E0E70000E82D00205F
:10B3E0000B010300616464725F69735F706167657C
:10B3F0005F616C69676E656428705F66732C20708E
:10B400006167655F6164647229000000705F667344
:10B4100000000000257320636865636B2066616926
:10B420006C656420696E202573282920776974680B
:10B430002076616C756520307825782E000000003C
:10B44000705F66732D3E705F617069006C656E00A1
:10B45000AC04030038B503000F484FF001054FF06E
:10B460000E04008805EB004009D061B119600C683A
:10B4700001B0A446BDE83040114618466047074B6E
:10B4800007A2009402E0054B07A2009408A100F077
:10B49000E6FC0E2038BD0000E82D0020C0000300AF
:10B4A000705F667300000000705F617069000000EB
:10B4B000257320636865636B206661696C65642031
:10B4C000696E202573282920776974682076616C5D
:10B4D000756520307825782E000000002DE9F041B8
:10B4E00028B1016819B1C969BDE8F04108470D4D9F
:10B4F0000D480024461B14270DE000BF04EB840018
:10B5000005EB8000016829B1C969884710B10120A5
:10B51000BDE8F081641CB6FBF7F0A042EED8002035
:10B52000F6E70000B02D0020C42D002004480121C2
:10B530004174007A08B10020704701207047000074
:10B54000F8360020012801D0032808D10449002240
:10B5500001284A7400D00020087402F0E7BD70474B
:10B56000F836002070B50246022801D0032A45D1E2
:10B57000234C207A002841D0012833D0022831D131
:10B5800020480023022A006802D0032A2AD11BE0A7
:10B59000E360017911B1012924D10DE0D0E90565FD
:10B5A000711B4FF48056B14200D33146294481616A
:10B5B0004569A9420ED015E00169491C0161426943
:10B5C00091420FD1237213E0E168491CE160082920
:10B5D00008D9E3602372022A0AD00D21FDF786FC08
:10B5E00002F04AFD607C28B1BDE8704000F0E4BF85
:10B5F0000021F3E7BDE8704002F098BD70BD000087
:10B60000F8360020242D00202DE9F84F3A4D040093
:10B610008B4628884FF00106DDF828A09846914611
:10B620004FF00E0106EB00401AD0B9F1000F1BD00D
:10B630002168002920D00921B8F1000F25D06268C7
:10B640005368B8FBF3F703FB1782002A21D02B4B7A
:10B650002BA2009135A100F002FC0920BDE8F88F73
:10B66000264B3DA2009102E0244B3DA200912FA168
:10B6700000F0F5FB0E20F1E7082100911F4B3AA2E4
:10B680002AA100F0ECFB0820E8E71C4B39A200914E
:10B69000E0E75846FBF7F5F9102798B14846FBF765
:10B6A000F0F9B0B1424659462046FBF7F0F9B8B17F
:10B6B000CDF800A0206843464A46C5685946204652
:10B6C000A847CBE7009728880C4B06EB00402AA23E
:10B6D0000CE000972888094B06EB00402CA205E0FF
:10B6E00000972888054B06EB004032A20FA100F01E
:10B6F000B6FB1020B2E70000E82D0020F8000300A0
:10B7000021286C656E202520705F66732D3E705F6A
:10B71000666C6173685F696E666F2D3E70726F67ED
:10B7200072616D5F756E6974290000002573206376
:10B730006865636B206661696C656420696E2025AD
:10B7400073282920776974682076616C75652030CC
:10B750007825782E00000000705F667300000000FE
:10B76000705F737263000000705F66732D3E705FE0
:10B77000617069006C656E00616464725F69735F1B
:10B78000616C69676E65643332286465737429007F
:10B79000616464725F69735F616C69676E6564336D
:10B7A00032282875696E7433325F7429705F737242
:10B7B00063290000616464725F69735F776974680C
:10B7C000696E5F626F756E647328705F66732C209C
:10B7D000646573742C206C656E2900002DE9FF41AF
:10B7E0001C46DDE90A7815460E46684600F0AAF8C0
:10B7F00046EA450141EA840141EA072242EA08415A
:10B80000009A00EB8200C0F80017BDE8FF812DE927
:10B81000FF411C46DDE90A7815460E46684600F0F1
:10B820009FF846EA450141EA840141EA072242EADB
:10B830000841009A00EB8200C0F80017BDE8FF81C4
:10B840002DE9FF411C46DDE90A7815460E4668469B
:10B8500000F094F846EA450141EA840141EA0722F2
:10B8600042EA0841009A00EB8200C0F80017BDE8E8
:10B87000FF812DE9FF411C46DDE90A7815460E4699
:10B88000684600F089F846EA450141EA840141EA48
:10B89000072242EA0841009A00EB8200C0F8001734
:10B8A000BDE8FF811CB5002100910B4601220191EA
:10B8B000FFF7C6FF1CBD1CB5002100910B460122FD
:10B8C0000191FFF7D6FF1CBD1CB500220B4600926C
:10B8D00011460192FFF7B4FF1CBD1CB500220B46B8
:10B8E000009211460192FFF7C4FF1CBD1CB5002158
:10B8F00000910B46012201911146FFF7A1FF1CBDEB
:10B900001CB5002100910B46012201911146FFF761
:10B91000B0FF1CBD13B50C46684600F021F8009935
:10B9200000EB8101D1F8002722F44032C1F8002752
:10B93000009900EB8100D0F8001741EA0441C0F8FB
:10B9400000171CBD0168202902D24FF0A0407047AB
:10B9500001F01F0101600148704700000003005022
:10B960000168202902D24FF0A040704701F01F016A
:10B970000160014870470000000300500168202961
:10B9800002D24FF0A040704701F01F010160014852
:10B9900070470000000300500168202902D24FF0D8
:10B9A000A040704701F01F0101600148704700008E
:10B9B0000003005001B56846FFF7D2FFD0F810052C
:10B9C0000099C84000F0010008BD01B56846FFF7C6
:10B9D000D5FF009A01219140C0F8081508BD01B5B6
:10B9E0006846FFF7D9FF009A01219140C0F8081579
:10B9F00008BD38B501240090684631B1FFF7A2FFB9
:10BA000000998C40C0F8084538BDFFF79BFF0099AE
:10BA10008C40C0F80C4538BD1CB5094C0144D4E934
:10BA20000034CDE900346C4606E000BF54F8203005
:10BA3000D3F81035401C08C28142F7D81CBD000065
:10BA40006C000300034908B5084400210160006848
:10BA5000009008BD0060004002494058012800D015
:10BA6000002070470060004030B5124B01460020B6
:10BA7000D3F81044224609E0157A854205D1401CCE
:10BA80000A28F7DB4FF0FF3030BD5268002AF3D1AF
:10BA9000421CF9D00872D3F810242AB152684A60C7
:10BAA000D3F81024516030BD0022C3F810144A604E
:10BAB00030BD000018380020F0B595B01C46154682
:10BAC0000F4608461A9E00F025FB182109A8FAF730
:10BAD000F4FC0E96CDE909540023082203A9384648
:10BAE00000F02DFB05980690BDF81000ADF81C0085
:10BAF000BDF81200ADF81E0000208DF8210003985B
:10BB0000082600F00300012802D0022818D032E0F5
:10BB100003983346850AC0F3C2008DF820000398CD
:10BB20000FA9C0F38314A200384600F008FB09A84F
:10BB3000009006AB22460FA9284600F047FA1AE00B
:10BB40000398840DC0F3C2008DF82000082C01D2A8
:10BB5000254600E0082533462A460FA9384600F05E
:10BB6000EEFA2E44641B09AB06AA29460FA800F082
:10BB70007FF9002CEAD1384600F0D2FA15B0F0BDBA
:10BB80007047012003F004BD084810B50178084A49
:10BB9000515C19B1001D01F0D3F802E00C3000F047
:10BBA000E1FFBDE81040002003F0F2BC382D00207A
:10BBB000742C002008B5034A00924023024AFFF784
:10BBC0007BFF08BD11EA0200183700200A4A01294C
:10BBD00002EBC00007D0022907D0032907D00429AF
:10BBE00007D000207047022070470420704700797A
:10BBF0007047407970470000F80B030010B5FFF75D
:10BC0000C0FF04210348FFF72FFF024901204872BB
:10BC100010BD00004C2D00202DE9F04F8DB0FCF739
:10BC2000C3FD18B100200DB0BDE8F08F7A4C4FF085
:10BC3000000BC4F818B4BFF34F8F60680290A5687A
:10BC4000D846284004EB800008E021680298814231
:10BC500001D86160E6E7284004EB80000C3002A9BF
:10BC6000FEF730FB0028F0D105AA029901EA05038E
:10BC700004EB8303491CDB6842F82030401C02912E
:10BC80000228F2D3059800F00300022802D0012810
:10BC90004ED0A9E005985022810D8946B2EB905F05
:10BCA00000D850210E4666F39F50059008315B483E
:10BCB00000F0E7F9070079D000F02CFA434608229B
:10BCC00005A9384600F041FA029908F1080A29400E
:10BCD000681A8000001D864223D94F4D0C3530B1C3
:10BCE000C2B204EB8101301A90460C3104E02946BF
:10BCF000F2B2002590462846C6B25346384600F0B8
:10BD000024FA0AEB08032DB1324629464FEA070010
:10BD100000F01BFA029909F1030001EB9000029078
:10BD20003BE004EB81015346324638460C31EFE7E5
:10BD30000598C0F38310062800D30620059960F308
:10BD40008911C1F38310801C05918100334800F0F4
:10BD500098F9070048D000F0DDF94346082205A90C
:10BD6000384600F0F2F908F1080800260FE00298C2
:10BD7000434600EA0501401C04EB810102900422C5
:10BD800038460C3100F0E1F908F10408761C0598FA
:10BD9000C0F38310B042EAD847B1D4F81054D4F8B5
:10BDA000180468B1384600F0BBF92FE01CE0687A4F
:10BDB000012804D12A6828463946126890476D68E0
:10BDC000002DF4D1384600F0ABF98DF800B068468C
:10BDD000FBF702F8D4F8180408B9029860609DF8DF
:10BDE0000000FBF71DF811E0D4F8104404E02168CE
:10BDF0002046896888476468002CF8D108480221E9
:10BE0000008801EB004007A100F016F8FCF7CCFC1D
:10BE100080F0010007E7000018380020800C0300C4
:10BE2000F82D00204261636B656E647320666C754B
:10BE3000736865640000000000231A4603F0E0B94F
:10BE400008B5012300926A4603F0DAF908BD1CB573
:10BE5000CDE9002302236A4603F0D2F91CBD3EB5AA
:10BE6000069C8DE81C0003236A4603F0C9F93EBD19
:10BE70002DE9F0470E4680461C46924608293ED8DA
:10BE800094F80C90002020731946104602F086F8B2
:10BE90000025B54206D218F805201AA12046FFF762
:10BEA0003DF903E019A12046FFF738F96D1C082D74
:10BEB000EFD317A12046FFF731F90025B54210D284
:10BEC00018F80570FAF7CEFA0068C05D10F03E0F62
:10BED00001D03A4600E02E220EA12046FFF71EF9BF
:10BEE00003E00DA12046FFF719F96D1C082DE5D3DD
:10BEF00001222146504602F033F884F80C90BDE848
:10BF0000F08700002025303278000000202020003B
:10BF10007C0000002563000020000000104810B5E0
:10BF2000FF218160002101604160C0F81814C0F851
:10BF3000141480F820140B4800F0F0F800280DD1FC
:10BF400009480A490A4B401AC108002003E000BF13
:10BF500023F82000401C8842FAD3002010BD0000C6
:10BF600018380020800C0300800C0300F80B03003D
:10BF7000C42D002002480349401AC0087047000041
:10BF8000800C0300F80B030013B56846FEF738FD7C
:10BF900008B100201CBD0248009950F831001CBDBA
:10BFA000F80B030070B508480125D0F8104480F85C
:10BFB000205405E065722168204649688847646816
:10BFC000002CF7D170BD0000183800202DE9FF4784
:10BFD00081460C9D00200C462F7B28739846164600
:10BFE0002946184601F0DAFF072E42D2DFE806F0B4
:10BFF00004090F161F2A360049462846FFF78EF817
:10C0000037E0494628462268FFF788F831E0D4E94E
:10C01000002349462846FFF781F82AE0A0680090EF
:10C02000D4E9002349462846FFF778F821E0D4E90F
:10C030000201CDE90001D4E9002349462846FFF773
:10C040006DF816E004F1080007C88DE80700D4E990
:10C05000002349462846FFF761F80AE004F108008A
:10C060000FC88DE80F00D4E9002349462846FFF7A2
:10C0700055F800222946404601F072FF2F73BDE8B3
:10C08000FF872DE9F041858A80462D1F4819C01C85
:10C09000B0FBF5F0C6B24046FEF737FE041E19D0DD
:10C0A0000020207101206071E58000272546761E62
:10C0B000C4F800800BE04046FEF727FE60B16179CE
:10C0C000491C6171286005467F1CC0F80080B7429A
:10C0D000F1D32046BDE8F081204600F002F80020B0
:10C0E000F8E72DE9F041457901466B1E002201E099
:10C0F0000968521C9A42FBD30F680146002605E0EE
:10C1000038460C68FEF723FE2146761CAE42F7D374
:10C11000BDE8F0810121001DFEF7CBBDFEF72FBE6B
:10C1200010B504460121001DFEF7E9FD10F0FF0FD8
:10C1300004D12046BDE81040FFF7D3BF10BD38B58D
:10C1400001240094FEF720FC38BD38B5002400948B
:10C15000FEF71AFC38BD0000064910B500204870F3
:10C16000091D0860BFF35F8F0349044800F050FACF
:10C17000002010BD2C2D0020680103000C3700208A
:10C1800008B500208DF800006846FAF725FEF1EEAC
:10C19000100A20F09F00E1EE100ABFF35F8F0849FC
:10C1A0004020C1F880029DF80000FAF739FE00F047
:10C1B000FDF908B141DF08BD20BF40BF20BF08BD69
:10C1C00004E000E0FAF76CBD20B1034909680160A2
:10C1D000002070470E207047540303002DE9FE43F2
:10C1E00006460D460846FFF7EFFF00287ED1804641
:10C1F000CDF80080CDF8048001244FF4A0708DF8B4
:10C200000060ADF80400CDF808808DF80240694662
:10C2100020202A6869DF404F40B100F03DFA024615
:10C2200038883E4904EB0040FFF70AFECDF8008055
:10C230008DF801408DF80280CDF80480CDF808809B
:10C240008DF80380694640202A6869DF40B100F01C
:10C2500023FA02463888324904EB0040FFF7F0FD2C
:10C26000CDF800808DF80060F720ADF80200CDF821
:10C270000480CDF80880694623202A6869DF40B130
:10C2800000F00AFA02463888264904EB0040FFF71E
:10C29000D7FDCDF80080CDF80480CDF808808DF86A
:10C2A00000804646694601202A6869DF40B100F0F7
:10C2B000F3F9024638881C4904EB0040FFF7C0FD43
:10C2C0004FF4B0600090019602966946A1202A685A
:10C2D00069DF40B100F0E0F902463888134904EB09
:10C2E0000040FFF7ADFD0096019600E011E00296D8
:10C2F0008DF800406946A0202A6869DF40B100F04F
:10C30000CBF9024638880A4904EB0040FFF798FD54
:10C310000020BDE8FE830000002E0020440A030038
:10C320008C0A0300D80A0300A4090300F0090300E3
:10C33000500903002DE9F0410446D0F8008060DF89
:10C340002168194D074641451CD92888022606EB6D
:10C35000004016A1FFF770FD2888424606EB00401A
:10C360001EA12368FFF773FDF006D0F80C012168C9
:10C37000800200F10050421A288825A106EB0040F7
:10C38000FFF75EFD012467B1384600F085F90246EB
:10C3900028882AA104EB0040FFF752FD3846BDE88B
:10C3A000F0812E480470F9E7002E0020496E737565
:10C3B0006666696369656E742052414D20616C6CDC
:10C3C0006F636174656420666F72207468652053C2
:10C3D0006F66744465766963652E00004368616E1C
:10C3E0006765207468652052414D207374617274D2
:10C3F000206C6F636174696F6E2066726F6D2030A0
:10C4000078257820746F20307825782E0000000081
:10C410004D6178696D756D2052414D2073697A6563
:10C4200020666F72206170706C69636174696F6EF1
:10C4300020697320307825782E00000073645F62D5
:10C440006C655F656E61626C652829207265747524
:10C45000726E65642025732E00000000AB2D002055
:10C4600030B51548ADF5017D0078002821D04FF496
:10C47000FA7500BFADF8005280A9684661DF38B197
:10C48000052816D00DF5017DBDE83040FAF708BC4F
:10C490006C460A497DA800F0BBF806E0D0E900210F
:10C4A000204690477DA800F0CAF87F980028E1D088
:10C4B000F4E70DF5017D30BDAB2D002058030300DE
:10C4C000F8B5134C2078C0B10120A07002F0ACF890
:10C4D000112814D0022002F0BFF800258DF800507A
:10C4E0006846FAF779FC11DF064625709DF80000D2
:10C4F000FAF796FC2EB13046F8BD0820F8BD0020B2
:10C50000F8BDA57002F034FE032002F0A5F8F6E7AE
:10C51000A82D00207CB5194C207808B108207CBDDE
:10C520000120A070002002F07FF8112819D000200F
:10C5300002F092F812480026006801908DF8006021
:10C540006846FAF749FC0F4901A810DF05000AD038
:10C55000002020709DF80000FAF762FC2DB12846FB
:10C560007CBD00207CBD0120F3E7A670667002F060
:10C570001BFE012002F070F8F3E70000A82D002058
:10C58000EC020300256C02000EB50749684600F076
:10C590003FF805E0D0E900108847684600F04FF802
:10C5A00002980028F6D10EBD080303000148007868
:10C5B00070470000A82D00200548817819B1007847
:10C5C00018B1FFF77DBF08207047FFF7A3BF000039
:10C5D000A82D00201FB568464BDF30B1052814D0C8
:10C5E00004B0BDE81040FAF75BBB084901A800F0B1
:10C5F0000FF806E0D0E900210098904701A800F06C
:10C600001EF803980028E6D0F4E71FBD740303006A
:10C61000016009684160AFF3008010B5D0E90021E6
:10C620005368994201D1002104E0D1E90034A342CA
:10C6300002D01946816010BD08314160F0E7816881
:10C6400000290BD0026892680A44826041684B68F6
:10C650009A4203D108314160FFF7DFBF7047000005
:10C660000C4A10B502F594730EE0991AC91001EB4B
:10C67000D171491002EBC1010C68844201D90B460B
:10C6800002E005D201F108029A42EED3002010BD6B
:10C69000486810BD8801030000B5FFF7E1FF0028DE
:10C6A00000D1014800BD000074010300405800287B
:10C6B00000D00120704708B5002242504058009039
:10C6C00008BDD0F80403084000D00120704740584E
:10C6D000002800D00120704708B500224250405881
:10C6E000009008BD08480068012110F0010F08D132
:10C6F0004FF0E020E02280F80024C0F88012C0F85B
:10C70000001102480160704700E100E01805004098
:10C710000649024600200B790BB1852070470A605C
:10C7200001220A7100224A7170470000882C002003
:10C7300004490120086004480168C1F30041002950
:10C74000FAD170470C00004018040040002802D0C5
:10C750000149800108477047910003002DE9F0412D
:10C760000E46804601F006F9204D0028404616D0BE
:10C77000FCF75AF8284490F858008009032802D0A2
:10C7800001280AD003E04046FFF714F928B103213D
:10C790004046BDE8F041FFF7BDB80221F8E701F0DF
:10C7A000F5F8002820D04046FCF73EF80446104F2C
:10C7B0004FF4807007EB840100EB8400D1F8102562
:10C7C00080B242F00102C1F81025FFF73BF9002EBC
:10C7D0000AD04046FCF728F855F82000002803D07E
:10C7E0000120A040C7F80403BDE8F0819833002081
:10C7F000006000402DE9FC41DFF8C080044608EBF2
:10C800000400002790F930001346C0170E46401C64
:10C8100001D008274FE0B0781946C0F34002204607
:10C82000FBF7DEFF0546401C44D0B07841071CD41E
:10C83000C0070DD068460094FFF792F8009900EB0E
:10C840008100D0F8001721F00201C0F8001707E0BE
:10C8500000217378204600910A460191FEF7D7FF28
:10C86000164920466431FEF7AAFAB078800718D539
:10C870001348317800EB8500D0F81025114B1A4091
:10C88000C0F810254FF47C524FF4403302EA0422E2
:10C8900003EA01410A43D0F810150A43C0F81025F5
:10C8A00009E008EB0500327810F8581F41EA8211C0
:10C8B000017000E004273846BDE8FC819833002071
:10C8C00000600040FFC0FCFF10B5FFF773F80028C0
:10C8D00000D0012010BD000070B5194D95F86A0018
:10C8E00008B1082070BD0020411E2A18401CC0B2AB
:10C8F00082F830103028F8D300242046FBF762FF7E
:10C90000641CE4B20C2CF8D30D490024E0204C66E2
:10C91000A1F868400B4981F8000401264020891FD6
:10C92000C1F88002C1F800014FF4BE70FFF78AF829
:10C930000549F007C1F8040385F86A60204670BD18
:10C940009833002006E000E000600040034890F8C3
:10C950006A00002800D001207047000098330020B2
:10C960000121B1EB507F01D10120704700207047B9
:10C9700038B50D4601F05EFB040014D000208DF8A0
:10C9800000006846FAF728FA207928B19DF80000DF
:10C99000FAF746FA112038BD0120256020719DF874
:10C9A0000000FAF73DFA002038BD10B501F042FB57
:10C9B000002802D000210160017110BD0149024828
:10C9C00002F00EBE04340020002000402DE9F041AA
:10C9D0000546007916460F4600EB40012D4A01EB53
:10C9E000C00102EB810494F82A1011B10820BDE8BF
:10C9F000F081294951F820102868FFF7B9FF08B1E4
:10CA00001120F4E739462846FAF750FA666038698B
:10CA1000206030004FF001062FD03F7F4FF48E7121
:10CA20002868FFF748FE4FF4A2712868FFF743FE1D
:10CA300028681A49C0F8041328684FEA4711000B08
:10CA400040B2002806DA00F00F0000F1E02080F884
:10CA5000141D03E000F1E02080F800142868000BAA
:10CA600040B200F01F0206FA02F14009800000F116
:10CA7000E020C0F88012C0F8001128680421C0F836
:10CA800000150020A061E06184F8290044F8140F2B
:10CA9000A675ACE704340020740003008000020097
:10CAA0002DE9F047054600790B4600EB400101EB0C
:10CAB000C000234901EB8004284600F043F810B180
:10CAC0001120BDE8F0874FF00008C4F82080A36073
:10CAD000626184F828804FF48E7647463146286894
:10CAE000FFF7E9FD28684FF00109C0F808902146DA
:10CAF000286802F011FD606800BBD5F800A00EE0C8
:10CB000094F8280008B10F2716E031465046FFF789
:10CB1000CDFD0028F4D02146504602F0FDFC216AEC
:10CB200060698142F1D331462868FFF7BFFD0028D4
:10CB3000F9D02868C0F80C90C4F814803846C0E7D3
:10CB400004340020007900EB400101EBC0000449EF
:10CB500001EB80004069002800D0012070470000F0
:10CB6000043400202DE9F047044600794FF0000915
:10CB700000EB400101EBC000254901EB8007206874
:10CB8000C0F80095786880B120682249C0F8081381
:10CB900020680121000B40B200F01F0291404009C3
:10CBA000800000F1E020C0F880112068D0F80C254A
:10CBB000D0F81485D0F80865D0F810554FF0FF3143
:10CBC000C0F81415C0F80C152068C0F80815C0F896
:10CBD0001015501C02D01046FEF764FEB8F1FF3F5E
:10CBE00002D04046FEF75EFE681C02D02846FEF7E3
:10CBF00059FE701C02D03046FEF754FE2068FFF745
:10CC0000D4FE87F82A90C7F80490BDE8F0870000AA
:10CC100004340020840202000149024802F08CBD65
:10CC200030340020002000402DE9F0410546164632
:10CC300000790F46154A00EBC00102EB810494F81D
:10CC4000201011B10820BDE8F081114951F82010E1
:10CC50002868FFF78DFE08B11120F4E73946284611
:10CC6000FAF75FF96660386920601EB1397F28469F
:10CC7000FDF7E8FA28680821C0F800150020A06137
:10CC8000E0610121606184F82010DCE7303400208D
:10CC9000780003002DE9F04704460E46007920494C
:10CCA00000EBC00001EB800517463046FFF758FE49
:10CCB00030B1204600F036F820B11120BDE8F087F1
:10CCC0001020FBE76F61AE604FF49076002731468D
:10CCD0002068FFF701FD4FF4AC7841462068FFF76C
:10CCE000FBFC2068AA686969C0F84425C0F84815AB
:10CCF000206801218160686878B9B146494620689A
:10CD0000FFF7E5FC064641462068FFF7E0FC0643D6
:10CD1000F4D000B10F27002068613846CEE700004C
:10CD2000303400200079054900EBC00001EB8000A1
:10CD30004069002800D001207047000030340020F6
:10CD40002DE9F04704460079274900EBC00001EBCC
:10CD5000800720684FF00009C0F80095786880B11E
:10CD600020682249C0F8081320680121000B40B256
:10CD700000F01F0291404009800000F1E020C0F85F
:10CD800080112068D0F80C25D0F81485D0F80865FB
:10CD9000D0F810554FF0FF31C0F80C15C0F814153D
:10CDA0002068C0F80815C0F81015501C02D01046B5
:10CDB000FEF781FDB8F1FF3F02D04046FEF77BFD54
:10CDC000681C02D02846FEF776FD701C02D0304663
:10CDD000FEF771FD2068FFF7E8FD87F82090C7F89F
:10CDE0000490BDE8F08700003034002010030200FA
:10CDF00010B590B1032814D10A480321008801EB33
:10CE0000004009A1FFF718F80220FBF73FFB0028BC
:10CE100007D0BDE81040F9F743BFBDE8104001F06E
:10CE20007BBF10BDF82D00204661737420616476CD
:10CE30006572746973696E672E00000000780028BF
:10CE400007D104483B21408876DF002801D0F9F75C
:10CE500027BF7047882B002070B58D88027900EBC2
:10CE6000C5042273C97BA41D012902D0022904D163
:10CE700001E0008800E040882080218860888142AD
:10CE80000FD92846A5DF0126A0B1112814D0FFF73D
:10CE900003FC02460A480BA1008806EB0040FEF79F
:10CEA000CFFFA179E079814208D92846BDE87040DA
:10CEB000FBF752BE6671F4E72671F2E770BD000021
:10CEC000C42D002073645F626C655F676174746376
:10CED0005F65786368616E67655F6D74755F7265C5
:10CEE000717565737428292072657475726E656436
:10CEF0002025732E000000007CB506468D88C8886A
:10CF000006EBC504A41D172800D2172021888142F2
:10CF100000D8084660800020207121882846B5DFAF
:10CF200050B1FFF7B9FB02460E480121008801EB22
:10CF300000400DA1FEF784FF6079002810D1306910
:10CF400000280DD01449D1E90201CDE90001ADF866
:10CF500002506088ADF80400326969463046904757
:10CF60007CBD0000C42D002073645F626C655F6748
:10CF7000617474735F65786368616E67655F6D7413
:10CF8000755F7265706C7928292072657475726E90
:10CF900065642025732E0000C4FF020048B1064AD4
:10CFA0000168914205D140680449401802D0012827
:10CFB00000D0032070470000DEC0ADDE02FEE10EAF
:10CFC0008A7D022A04D90289CB881A44D21C0281A4
:10CFD0004289C988511AC91E418170472DE9F04123
:10CFE0000D460221904600F58056298000F1080484
:10CFF000144F1BE031462046FCF7C2FD40B1B8F1AA
:10D00000000F02D0012288F80020022816D004E088
:10D01000A0687969884200D97861288861880844C5
:10D02000C01C2880608804EB80040C343146204604
:10D03000FCF7B9FD0028DDD1BDE8F0814FF4806038
:10D040002880F9E7E02C002008B500210091014676
:10D050000823024A0248FEF7D7FA08BDA8000300D9
:10D06000B02D002008B50020009004480823044A91
:10D0700001680448FEF7C8FA08BD0000082D00202A
:10D08000A0000300B02D00202DE9F05F0025DFF89F
:10D090000891DFF808B12C464FF00308AA462F4646
:10D0A000D9F80C0000EB07363046FFF777FF78B36E
:10D0B000012847D0032862D100204FF4806200BFCE
:10D0C00056F82010491C0ED004EB84010BEB8102B2
:10D0D000A8F10100566003221FFA80F80BF8212006
:10D0E000641CA4B24BE0401C9042E9D32C48016878
:10D0F00079B104EB840102200BF821000BEB8101D4
:10D100004E600881254828304480641CA4B205E0A4
:10D1100007E00221066081804FF0010A45F0010519
:10D120002DE004EB840100220BF821200BEB8101A0
:10D1300001F110024E6030460831FFF74FFF45F015
:10D140000205CDE7BAF1000F0CD0022004EB8401F8
:10D15000134A0BF821000BEB810112684A60641C32
:10D160000881A4B20E480022011D06603046FFF778
:10D1700035FF0B48808802280CD0082005437F1C0F
:10D18000BFB2032F8CD3B8F1020F00D20025E8B252
:10D19000BDE8F09F0420F1E7B02D002034360020D8
:10D1A000082D002001494978FAF752BC0C2C0020C8
:10D1B000002101F0B1BF30B585B00C4605218DF8D6
:10D1C00000101546ADF80200FCF732FFADF8040080
:10D1D0006846CDE90245FBF71FFF05B030BD0000F2
:10D1E00070B5054D06460024304655F82410884792
:10D1F000641C042CF8D370BDF4FF02003EB5104D42
:10D20000002400BF05EB041002F034FD641C022C66
:10D21000F8D30124502002210094CDE901100849DF
:10D22000084BB039A02201F1A00000F0E9FB08B1E1
:10D2300003203EBD0348401E847000203EBD000018
:10D24000D8320020F92B002000F06CB900F06CB946
:10D2500070B504460025C168184A284602EB001341
:10D260009B688B4202D102EB001003E0401C0228B5
:10D27000F4DB00202178082904D0092908D01329DB
:10D2800014D112E0617A89B980B102F003FD0DE09A
:10D29000617A59B950B100218160817B41F002016E
:10D2A000817307490120087003E001252046FFF73C
:10D2B00097FF2846BDE8704000F0C4BFD832002078
:10D2C000F82B002000F0E5B908B513889B00009307
:10D2D0006B4600F05FF908BD002300F05BB938B57C
:10D2E00005460024204609E08178284600F080F8B1
:10D2F00010B1052800D003240098401C0090694616
:10D30000284602F0A3FC0028EED134B9284600F0EC
:10D31000C4F910B1072802D00324204638BD0724E1
:10D32000FBE71346002200F069B900002DE9F04741
:10D330001F0015460E46814604D0072E05D0082E44
:10D3400016D102E00E20BDE8F0878DB1022D0FD876
:10D3500000F0AEF960B14FF000083146484602F0E7
:10D360005BFC041E06D0207BA8420DD00F20EAE70C
:10D370000720E8E7FF214FF6FF7002F04DFC041E86
:10D3800006D0A0F80090A670607BFF2802D00CE0C9
:10D390001120D8E72946154800F004FB0146204635
:10D3A0006173FF2913D04FF001082573617B0F488B
:10D3B00000F046FB02000DD0ABB23146384600F01B
:10D3C00007FAB8F1000F0ED0082E05D00BE002F0DE
:10D3D00051FCDDE70320B6E738886FF0050101EB6B
:10D3E0008000796888800020ADE70000C832002006
:10D3F00070B5002402F010FC05000BD0686820B165
:10D4000000F06FF9040000D00324284602F042FC2B
:10D41000204670BD052070BD70B515460C46072925
:10D4200003D0082C01D0072070BD02F0F5FB28B115
:10D4300005808470BDE8704002F0ACBB052070BD73
:10D440007CB50D46072903D0082D01D007207CBDEF
:10D45000002602F0E1FB040002D0606810B11CE07D
:10D4600005207CBD617B0F4800F0EAFA02004FF016
:10D470000000009001908DF8025010D0237B2946C7
:10D48000684600F03DF9684602F072FB211D6846CF
:10D4900000F010F90646092801D030467CBD032073
:10D4A0007CBD0000C83200204FF6FF714180014969
:10D4B00009680847DCFF020030B587B01748FBF762
:10D4C00037FF10B1032007B030BDFBF753FE08B1A2
:10D4D0008620F8E700F0CEF9002002904CF2070415
:10D4E00003900EE0694604A8FBF7ECFE00988088E4
:10D4F000A0F5404085B204A8FBF7A4FE284600F042
:10D5000075F902AA04A92046FBF7C3FE0028E9D05A
:10D510000349012008700020D5E70000299002008F
:10D52000EC2B002000F088B900F08CB970B586B003
:10D5300014460E46054600F03BF940B105F5404063
:10D5400080B20F4A6946FBF7A4FE40B902E0012011
:10D5500006B070BD03A96846FBF7B4FE08B1002011
:10D56000F6E7A570039840882080049860600398CF
:10D570008088A0F5404030806846FBF763FEE6E710
:10D58000F02B0020024800214160816070470000BC
:10D59000EC2B0020F0B587B01D46144607460E461A
:10D5A000FF280AD8084600F003F930B103AA314633
:10D5B000384600F0E5F840B902E0072007B0F0BDBA
:10D5C00001A903A8FBF77EFE08B10520F6E7A670C7
:10D5D00001984088208045B18200286890420BD392
:10D5E00002996068F8F742FF01E00298606003A8C2
:10D5F000FBF728FE0020E1E70420DFE77FB586B0D7
:10D600001E460D460446FF282AD8A87800F0D0F818
:10D6100030B304F54040ADF80000A87803AA00F547
:10D620004040ADF802006868019028880290A9780F
:10D63000204600F0A5F80528089813D010B108A8D6
:10D64000FBF7A4FE694603A8FBF760FEB0B107280C
:10D650001DD0082819D00E2817D003200AB070BD9D
:10D660000720FBE728B108AA694603A8FBF759FE83
:10D67000ECE7694603A8FBF750FEE7E71EB1314629
:10D6800003A8FBF716FE0020E8E71120E6E7862056
:10D69000E4E74FF6FF7000F0A9B810B5FF2801D9F4
:10D6A000072010BD00F0A8F800F02EF8002010BDF3
:10D6B00000F0F4B870B504460D46807800F078F8B4
:10D6C00058B121882846FBF749FE002804D00728D6
:10D6D00005D0092800D0032070BD072070BD86202A
:10D6E00070BD01B56846FBF751FE002800D003204D
:10D6F00008BD00000149C978FAF7AAB90C2C00202E
:10D700009BB200F065B8000070B51B4D8AB00020D8
:10D71000687000904FF6FF760190304603E0204697
:10D7200000F07CF8204600F087F80446B0421DD097
:10D7300004F5404080B26A4602A9FBF7B2FD0A2810
:10D74000EDD004F5404080B2FBF7D4FC08280FD0A0
:10D7500000280BD005461422084905A8F8F786FED4
:10D76000ADF8184005A80795FFF79EFE0AB070BDFA
:10D7700001206870FAE70000EC2B0020E0FF0200B7
:10D780007CB5054616460C46084600F011F8002008
:10D79000009005F54045019004F54044A8B2A1B2BF
:10D7A0006B463246FBF76EFD002800D005207CBD9D
:10D7B00007280BD0012809D0082807D0052805D054
:10D7C000062803D0042801D00020704701207047AC
:10D7D00010B503EB83034FF6FF7404EA0313817063
:10D7E000DB1C99084260018010BD00000149FBF775
:10D7F00073B80000F832002010B50446A0F57F4051
:10D80000FF3807D004492046FBF766F8A04201D153
:10D81000012010BD002010BD1833002010B50446B3
:10D82000044900F02BFE03492046BDE8104020319A
:10D8300000F024BEF83200200149FDF77DB9000058
:10D840001833002070B50A49FDF776F904464FF603
:10D85000FF7507E000F02CF838B105492046FDF7C8
:10D860006BF90446AC42F5D170BD204670BD000096
:10D87000F832002010B508484021F8F71EFE4FF49A
:10D8800080742146044800F0ADF921460248BDE805
:10D890001040203000F0A6B9F8320020FF2803D84D
:10D8A0000146024800F0CDB900207047F832002050
:10D8B000FF2803D80146024800F0C3B90020704792
:10D8C0001833002010B50C46FCF71EF8FF2804D0D2
:10D8D000024900EB400021F8204010BD2831002013
:10D8E0001CB500F059F908B1F9F7DAF900200090F9
:10D8F00001909DF8000020F0720040F001003030EF
:10D9000020F080008DF8000007208DF80100102025
:10D910008DF802009DF8030040F003008DF803002D
:10D920009DF8040040F003008DF80400684600F004
:10D93000EDFA08B1F9F7B4F9064800F0D1FA08B1E8
:10D94000F9F7AEF90448FBF7F3FC002801D0F9F72A
:10D95000A7F91CBDA1DA0200259002000068012889
:10D9600005D0022803D0042801D0002070470120F0
:10D97000704700000449084490F93000082801DB92
:10D980000120704700207047983300200449084464
:10D9900090F93000082801D201207047002070471C
:10D9A000983300202DE9F0410F46060026D030685C
:10D9B00020B3706810B3FF2400251CE0294670686E
:10D9C00000F017F948B1FF2C00D12C46281B401C51
:10D9D000B8420ED12046BDE8F081FF2C06D108E008
:10D9E0002146304600F040F8641CE4B2AC42F7D364
:10D9F000FF246D1CEDB2B068A842DFD8FF20EAE733
:10DA00002DE9F0410400DDE90705069E16D0A9B115
:10DA1000A3B100FB05F7974210D8C21DB6EBD20F99
:10DA20000CD358B155B1E5602160C4E9013081B231
:10DA3000184600F0D7F80020BDE8F0810720FBE78A
:10DA400070B504000D460DD0206858B1606848B12B
:10DA5000FF2D07D000F0F5F820B1E168206805FB44
:10DA6000010070BD002070BD70B504000D4611D0DE
:10DA7000206800280ED0606800280BD0FF2D09D048
:10DA800000F0DFF8002805D029466068BDE8704046
:10DA900000F0E3B870BD002901D001F061B9704712
:10DAA000F8B5044600781E4D03260E281DD2DFE887
:10DAB00000F0071C0F1C1D1C24351C331C352E3593
:10DAC000288818A106EB0040BDE8F840FEF7B4B97D
:10DAD0006088F9F78DFF0246207A009028886388D5
:10DAE00006EB00401AA1FEF7BAF9F8BD002000903D
:10DAF00060886946FFF7CFFFF8BDFBF71DFB0828DC
:10DB0000FAD00028F8D0BDE8F840F9F7C9B8BDE868
:10DB1000F8400020F8F7E2BF2069F2E7A068F0E7DC
:10DB2000F82D0020436F6E6E656374656420746F1A
:10DB300020612070726576696F75736C7920626FF1
:10DB40006E646564206465766963652E000000007C
:10DB5000436F6E6E656374696F6E20736563757273
:10DB600065643A20726F6C653A2025642C20636FDF
:10DB70006E6E5F68616E646C653A20307825782C33
:10DB80002070726F6365647572653A2025642E009B
:10DB9000FBF71EBAFBF71CBA10B5FFF78DFC88B96E
:10DBA000FFF72CFB70B901F0DDF858B901F0F8F976
:10DBB00040B9FBF745FE28B9FBF72AFF10B9FCF77F
:10DBC000A7F908B1032010BD05484FF6FF71818009
:10DBD00000218160417001210170002010BD000012
:10DBE000FC2B0020002803D0C91DC908F8F765BC2C
:10DBF0007047002809D001F0070301229A40D2B2F1
:10DC000000EBD1001146FCF75BBD70472DE9F041F8
:10DC10000D46060013D0002401270EE004F0070093
:10DC200007FA00F0C1B206EBD400FCF749FD10B1D1
:10DC30002046BDE8F081641CA4B2AC42EED3284675
:10DC4000F7E740B100EBD10001F0070200780121B5
:10DC50009140084000D001207047F8B50400C1F39E
:10DC6000C70501F007014FF0010000FA01F0C6B24C
:10DC70000FD0605D30420CD000208DF80000684667
:10DC8000F9F7AAF8605DB04360559DF80000F9F718
:10DC9000C7F8F8BD2DE9F041044686B00127808819
:10DCA000FCF704F96080207800263F4D082808D052
:10DCB000092820D04FF6FF780A2829D00B2853D105
:10DCC00058E0607A10B1012809D04DE0A86830B161
:10DCD000E168814203D1AE60A088A88016E0687830
:10DCE000E8B3A088A98888423ED1207A06283BD193
:10DCF00000F08CFA38E0607A88BBA86878B3E168F5
:10DD0000814231D1AE60E868401EE860E6602BE0F9
:10DD1000A878E8B14046FFF799FA4146404517D147
:10DD20000846FFF791FA404512D1AE7014216846BB
:10DD3000F8F7C3FB0C208DF80000ADF80480ADF8B7
:10DD4000028000272046FBF743F96846FBF740F9BD
:10DD5000687838B1A088A988884203D100E003E040
:10DD600000F054FA002F1CD006B02046BDE8F04168
:10DD7000FBF72EB9A8780028F6D0AE7014216846BB
:10DD8000F8F79BFB0D208DF80000ADF80480ADF88E
:10DD90000280A06802902046FBF71AF96846FBF75C
:10DDA00017F906B0BDE8F081FC2B00200349097883
:10DDB00009B1FCF729B9082070470000FC2B0020AE
:10DDC0002DE9FF4F2A4883B09946007892468B464A
:10DDD000B8B14FF6FF763046FFF738FA804600209C
:10DDE0000090244801AA062100680190CDF808D0CF
:10DDF0004046FFF769FA00256C1E3746072804D015
:10DE000017E0082007B0BDE8F08F0520FAE70020F2
:10DE10000090A84201D305464746A04201D20446DD
:10DE200046464046FFF712FA804601AA0621FFF750
:10DE30004BFAD8B10528EAD0A8F57F41FF3901D0C7
:10DE40000320DFE70399002001B10F80BBF1000F31
:10DE500001D0CBF80050BAF1000F01D0AAF8006051
:10DE6000B9F1000FCED0C9F80040CBE70098D0E759
:10DE7000FC2B00200400030070B5184E86B03078EB
:10DE8000D0B10120B0704FF6FF742046FFF7DEF9E5
:10DE90000546A0421DD10020B07014216846F8F755
:10DEA0000CFB0C208DF80000ADF80440ADF80240EA
:10DEB0006846FBF78DF80EE0082006B070BD00BF85
:10DEC000FFF774FF08B10320F7E72846FFF7BEF914
:10DED0000546A542F4D10020EFE70000FC2B00200E
:10DEE000084A117821B1D178032903D3042070475F
:10DEF00008207047044B43F82100491CD1700020D2
:10DF000070470000FC2B00203833002003490978BB
:10DF100009B100F079BF082070470000FC2B0020F9
:10DF2000002801D0FBF754B8704770B50D000446C7
:10DF300002D10020F8F7B4FE14B90020F8F7B0FEC3
:10DF40002878207069886170090AA170A988E17039
:10DF5000090A2171E8886071000AA07170BD000093
:10DF600010B50C46017A052908D0407A38B1084826
:10DF700008A102682046FDF7D1F800E01AB106A119
:10DF80002046FDF7CBF82046BDE81040FDF7D3B89A
:10DF9000842D0020257300000D0A000038B5C388C9
:10DFA0000D46044633B114A0009015A216A12846D0
:10DFB000FDF7B4F8217A05291CD0607A48B1A08811
:10DFC000FDF704FE164951F8202016A12846FDF75A
:10DFD000A5F8A0880021FDF7D7FF03461049207A55
:10DFE000143951F8202001B02846BDE830400EA178
:10DFF000FDF794B838BD00001B5B306D00000000D9
:10E000001B5B313B33316D0025734C6F67732064AC
:10E01000726F70706564202825642925730D0A00CD
:10E02000842D0020257300003C25733E2025733A83
:10E03000200000000349884201D1034870470020B6
:10E040007047000000200040902C00200146054849
:10E0500010B50068FCF7A3FD04461C21F8F72DFA63
:10E06000204610BD98000300014602480068FCF7F6
:10E07000B7BD000098000300034802490068FCF7A0
:10E0800099BD0000282D002020010300F0B5254D8A
:10E09000254E85B004460027686828B921493068B4
:10E0A0000831FCF792FD686001460078072817D216
:10E0B000DFE800F0160408080E0E12002046FBF7F9
:10E0C000FFFF02E0204601F06FFE040028D008E0C8
:10E0D0002046FAF7DFFDF8E72046FBF75BFAF4E7A6
:10E0E0000F2414216846F8F7E8F9A4F5E8501D3824
:10E0F00000D10024019469466868FAF7ADFE6846CD
:10E10000FAF7E4FE07496F60002408313068FCF735
:10E1100051FD044801210C30FCF7F1FD0028BBD172
:10E1200005B0F0BDE02C0020980003002DE9F0417F
:10E13000234C0025234E207A012730B92248311D77
:10E140000068FCF742FD306038B10220207231686F
:10E15000087928B101281ED116E06560BDE8F0817C
:10E16000D1E90503C01A4FF48052904200D3104603
:10E17000B7EB900F01D2820800E001220869C9685C
:10E180001844194429DF03E0D1E90301084428DFDA
:10E1900058B1112812D003213068FAF7A7FE257272
:10E1A0006560BDE8F041FFF767BF207C0028D5D14E
:10E1B000BDE8F04100210220FDF7D4B92772CDE778
:10E1C000F8360020242D00202001030010B5012185
:10E1D0000448FCF77AFD002803D1BDE81040FFF7A2
:10E1E00055BF10BDEC2C002010B5074C201DFCF7CE
:10E1F0005DFD002806D1607C002803D1BDE81040F9
:10E20000FFF794BF10BD0000F8360020084910B594
:10E2100000231A46A1F10800FFF7D2FD30B105280E
:10E2200004D0002002490C39487010BD0120F9E7E4
:10E23000082C002010B510461A46F8F717F90020F0
:10E2400010BD00002DE9F0471B4F824600263878AC
:10E2500086B0002821D00024DFF86080A14600BFEE
:10E2600008EB0415A87B810702D410EA0A0F1BD023
:10E270000126284601F08EFCB0B14FF6FF71ADF8D3
:10E2800002102988ADF80410862809D007218DF8DE
:10E29000001002906846FEF7A3FF06B0BDE8F087C5
:10E2A00006208DF80000F5E7641C022CD8D3002E60
:10E2B000F3D187F80090F0E7F82B0020D832002047
:10E2C0002DE9F04707461E481C46154600780E46C5
:10E2D00070B185B17CB1DFF86C804FF00009A08887
:10E2E00002282BD200EB800118F8210010BB19E0A6
:10E2F0000220BDE8F0870520FBE720681FB1818878
:10E300003A8891420ED11EB101883288914209D1DA
:10E3100080682860206868600A4828300089288161
:10E320000020E6E7A088214600F05EF80028E4D14E
:10E33000C4F80090A088401CA080D0E70A20D8E74D
:10E34000002D002034360020F8B505464068244FE3
:10E350000C46002648B32349CA68824225D8096979
:10E36000814222D3FCF708F8F8B12889398988421C
:10E370001BD1D5E900018A68904216D10020A7F18F
:10E38000280200BF00EB800302EB83035B688B4233
:10E3900005D203F580538B4201D9208011E0401C47
:10E3A00080B20228EED30020F8BD268000960AE055
:10E3B000009829688068884205D10098686038898B
:10E3C00028810120F8BD2088694600F00DF800285A
:10E3D000EED12088401C80B220800228E6D3E2E7FC
:10E3E0005C360020B02D002070B50E4600EB800199
:10E3F000134800EB81004468306804F5805518B17B
:10E40000418800EB810411E0083410E029462046E1
:10E41000FBF7B6FB20B1012805D0022807D10DE09B
:10E420000120346070BD608804EB80040C34294600
:10E430002046FBF7B8FB0028E8D170BD002070BD76
:10E440003436002038B50C460021009101460423E3
:10E45000074A0848FDF7D8F808B10E2038BD064A2B
:10E4600004EB840102EB810101200874002038BD17
:10E470009C000300B02D0020343600200A46FF28FF
:10E4800003D801461046FFF7E8BB704708467047BF
:10E490001E4810B50078002837D01C481C49183099
:10E4A00000F0A9FA81B21B48F9F717FE174818497E
:10E4B000183000F0A0FA81B21648F9F70EFE1348A2
:10E4C0001349183000F097FA81B21248F9F705FEA7
:10E4D0000E480F49183000F08EFA81B20D48F9F756
:10E4E000FCFD0A480A49183000F085FA81B2094853
:10E4F000F9F7F3FD05480649183000F07CFA81B2BF
:10E50000BDE810400348F9F7E8BD10BD882B002096
:10E51000E42F0020882E002070B5012670044FF0F3
:10E52000E0210025C1F88001084C4010C4F84803E0
:10E53000C4F8080366602F20FEF708F9A660044CB3
:10E540002F20A560FEF702F9A57070BD00100140F4
:10E55000B82C002070B5054688690C4600284FF499
:10E56000847128460AD0FEF7A6F8D5F81805626A25
:10E57000E1688854606A401C606270BDFEF79BF8D9
:10E58000D5F8180570BD1FB501238DF80030CDE911
:10E590000121D0E90012684690471FBD1FB5012335
:10E5A0008DF800308DF808100192D0E9001268460D
:10E5B00090471FBD10B50446064841792046F9F73B
:10E5C00047FA002804D12046BDE8104000F06CBA9C
:10E5D00010BD0000D42B002038B50021012548B122
:10E5E00001280CD0032809D1FEF77CF8BDE838409B
:10E5F000FCF748BD4FF0E020C0F8805138BD8DF8E1
:10E6000000106846F8F7E8FB064C207808B9FCF7DC
:10E610001DFDE068401CE060A5709DF80000F8F763
:10E62000FFFB38BD843300203EB5044609496846E7
:10E63000FDF7EEFF08E000BFD0E90021204690473B
:10E6400030B16846FDF7FBFF02980028F4D13EBDCB
:10E6500011203EBDF00203003EB50446084968465D
:10E66000FDF7D6FF07E000BFD0E900212046904724
:10E670006846FDF7E4FF02980028F5D13EBD000092
:10E68000FC0203002DE9FC4104460C3000278046C3
:10E69000FBF7DEFC4FF6FF750646A842208803D143
:10E6A000FBF7C6FC064602E03146FBF7ABFC2088D0
:10E6B0000022012100F0C6F8AE4212D06A460721BE
:10E6C0003046FEF709FE60B9019D95F844003435E7
:10E6D000C00705D1414605F11200FBF77EFC00B1F1
:10E6E0002F46002320881A46394686DF05000BD0C6
:10E6F000002320881A46314600F088F820882946F1
:10E7000000F002F9BDE8FC81002FFBD10023208836
:10E710001A46314600F07AF82088002241F20601BC
:10E72000FAF76EFBEEE700002DE9FC411D46089C60
:10E7300016460F46804644B16B46012207213846F3
:10E74000FEF7F4FD112801D010B10320BDE8FC81D3
:10E7500050210198F7F7B1FE019806700198E56025
:10E76000343020600198183020610198401C6061AD
:10E770000748E061019940461131FBF71BFB002877
:10E78000E3D107213846FEF75BFE0528DDD0DDE743
:10E7900044330020002835D00278910701D41106B7
:10E7A0002FD4C2F3021104292BD8930703D50329D0
:10E7B00001D1110625D5437881788B4221D8072BCA
:10E7C0001FD310291DD8C1784B071AD400794307ED
:10E7D00017D40B0715D4030713D4D2074FEAC1721D
:10E7E00001D042B10FE062B989070AD4C10708D14C
:10E7F000800706D407E0890705D4C10703D1800745
:10E8000001D40020704701207047000070B50C460D
:10E8100005466AB1002B12D009480122C17828466A
:10E82000F9F72EF921462846BDE87040FBF7EABB10
:10E83000002B04D0BDE870400846FBF7E5BB70BD77
:10E840000C2C0020F0B5174D14460F460A4685B033
:10E8500006462978F9F714F9002F1FD00CB10122D0
:10E8600000E0002269783046F9F70AF9012C17D048
:10E870000022A9783046F9F703F90022E9783046FA
:10E88000F9F7FEF8142208496846F7F7EFFDADF8EE
:10E8900002608DF808406846FAF7B0FB05B0F0BD9D
:10E8A0000122E6E70C2C00201800030010B586B00A
:10E8B000044614216846F7F700FE04208DF8000096
:10E8C000ADF802406846FAF799FB06B010BD0000AB
:10E8D00002498969002900D0084770479430002018
:10E8E00030B585B00C460546142206496846F7F750
:10E8F000BDFDADF8025068460294FAF75BFB05B027
:10E9000030BD000054FF020030B585B00C4605460E
:10E91000142206496846F7F7A9FDADF8025068468B
:10E920000294FAF76BFB05B030BD00002C00030029
:10E930000348417881F0010141700248F9F7E8BBD2
:10E94000882B0020882E002070B515480124512105
:10E9500064258460C0E9001504730146114800F085
:10E960003FF80F488C211030002601604FF496715B
:10E9700041600A218160067301460A48083000F0B0
:10E980002FF807484FF4FA7120300560C0E90114F0
:10E9900006730146BDE870400248103000F020B810
:10E9A000C42F0020902B002010B503680A688968E6
:10E9B0009C1A8C4202D9591A016010BD01210260D3
:10E9C000017110BD10B54B68026889689C1A8C42B1
:10E9D00002D91144016010BD00210360017110BD16
:10E9E0000A7B1AB149680160002102E009680160F0
:10E9F00001210171704710B50446007900282046B6
:10EA000002D0FFF7DFFF01E0FFF7CEFF206810BD67
:10EA100070B50D4C0020D2B22070201D0B4D037834
:10EA2000EB5C1BB1001DFEF735F902E00C30FEF780
:10EA300037F808B1F8F734F96078002802D0217867
:10EA40000029FAD070BD0000342D0020742C002065
:10EA50000348002201490079F8F7B4BFB5E5020088
:10EA6000D42B00207CB50E490E4C0022D1E90001C8
:10EA7000CDE900016946A088FEF753FC4FF6FF750B
:10EA800007E00846FEF7E2FBA08000226946FEF799
:10EA900048FCA188A94201D01128F2D17CBD000018
:10EAA000A8FF0200E02B002070B586B006460125C5
:10EAB0000024FBF749F8112812D005DCF0B1062834
:10EAC00028D0082808D125E0A0F54051023907D008
:10EAD000A1F54071FF3924D001463046FFF700FF11
:10EAE0002A46124D30462979F8F7CAFF697906B0EF
:10EAF00022463046BDE87040F8F7C2BF14220C49E8
:10EB00006846F7F7B3FCADF8026001246846FAF7EF
:10EB100051FAE5E700253046FBF78AFAFAF76AFF73
:10EB2000DEE73046FBF790FDDAE70000D42B00204B
:10EB30007CFF02002DE9F0410746806A14468846B2
:10EB4000C8B3002531E000BFB96A05EB450001EB11
:10EB50008006B088801CFE2802D90C20BDE8F08118
:10EB60002288401C08F8020020881622401C80B22F
:10EB7000208008F800202088401C80B2208000EB14
:10EB80000801308800F052FE2188084480B22080BD
:10EB9000B28842B1B16871B14044F7F767FC208890
:10EBA000B188084420806D1CEDB297F82C00A84273
:10EBB000CAD80020D2E7FFE70720CFE730B59DB0E5
:10EBC0004E481A9000241AA94D48FCF7C2F908B122
:10EBD000F8F766F803208DF86C0014216846F7F703
:10EBE0006CFC1BA802909DF80C00012520F00F0082
:10EBF000401C20F0F00010308DF80C009DF80D0046
:10EC0000009420F0FF008DF80D009DF80E008DF8A7
:10EC1000045020F0FF008DF80E009DF80F006946AB
:10EC200020F00F00401C20F0F00010308DF80F0095
:10EC30009DF8100020F0FF008DF810003048783863
:10EC4000F9F7E6F908B1F8F72BF8142105A8F7F75A
:10EC500034FC9DF82100059420F00F00401C20F0AA
:10EC6000F00010308DF821009DF822008DF818502A
:10EC700020F00F00401C20F0F00010308DF8220032
:10EC80009DF82300079420F0FF008DF823009DF8E5
:10EC9000240005A920F00F00401C20F0F0001030E7
:10ECA0008DF8240064208DF8200015482838F8F7E6
:10ECB000F7FD08B1F7F7F4FF40210AA8F7F7FDFBCD
:10ECC00010A10AA8F9F727FA9DF8640020F00F00B8
:10ECD000401C20F0F00010308DF864009DF86500B5
:10ECE00020F0FF008DF865000AA8F8F723FF002840
:10ECF00001D0F7F7D5FF1DB030BD0000C5C102003F
:10ED0000002F00204E6F7264696353656D69636FF5
:10ED10006E647563746F720010B50020F9F7B6FB6E
:10ED200008B1F7F7BDFFF9F70BFB08B1F7F7B8FF2C
:10ED300033DF002803D0BDE81040F7F7B1BF10BDA6
:10ED400010B500F0ABF80548002203494078BDE853
:10ED50001040F8F737BE000025A50200142C002053
:10ED600000F016B910B51148FAF747FB0F48401CE0
:10ED7000FAF743FB0D48801CFAF73FFB0B48C01C19
:10ED8000FAF73BFB0948001DFAF737FB0748401D1F
:10ED9000FAF733FB0548401E8179182903D0012179
:10EDA000C171002010BD032010BD0000152C0020F3
:10EDB00010B50078114C0A2813D004DC082810D0B4
:10EDC00009281AD10DE00B280BD0132815D10022E9
:10EDD0000B49A079F8F7F6FD00220A49A078F8F768
:10EDE000F1FD002206496079F8F7ECFD6078BDE896
:10EDF000104000220349F8F7E5BD10BD142C002097
:10EE0000B1D1020025A5020070B50B4C05004FF0F2
:10EE100001060CD0FFF7BEFC58B1286820612879A4
:10EE2000207504F11000A0602670002070BD002045
:10EE3000F9E7072070BD0000142C002010B504462F
:10EE40000078052802D0122821D105E06088A16849
:10EE5000BDE8104000F060B90F480021806880B123
:10EE60000D48237A1030007800F0010203B101232D
:10EE70009A4206D3627AC0F3400002B10122904266
:10EE800000D20121608801230022FBF7A9FA204665
:10EE9000BDE81040FAF7C0B8142C002030B5044685
:10EEA000008885B014284FD00ADC11282CD01328F4
:10EEB00028D134F8040FF8F79BFD01282FD038E053
:10EEC000192847D01A281DD1A088FEF76BF9002811
:10EED00018D1A088F8F766FD0028A0884BD02A49F1
:10EEE00000220978F8F7CCFD02208DF80000A088F8
:10EEF000ADF8020000208DF808008DF80900684682
:10EF0000FAF77CF805B030BD207A3D2804D04FF4E4
:10EF10008851A088002224E041F23D01F9E72079E0
:10EF2000C00701D0012200E0022220880121FFF762
:10EF300089FC34F8045B142214496846F7F796FA02
:10EF4000ADF802500294DAE705B0201DBDE830406C
:10EF5000FFF798BB217A201D41B14279008802F069
:10EF6000030205B0BDE83040FBF796BA05B0BDE836
:10EF70003040F8F713B805B00122BDE8304041F247
:10EF80000601F9F73DBF00000C2C002054000300DF
:10EF90000A7802490979F8F773BD00000C2C0020AB
:10EFA00010B51448FAF720FA1248401CFAF71CFA78
:10EFB0001048801CFAF718FA0E48C01CFAF714FA29
:10EFC0000C48001DFAF710FA0A48017818290FD0EA
:10EFD000417818290CD08178182909D0C1781829CE
:10EFE00006D00179182903D001214171002010BDFC
:10EFF000032010BD0C2C002070B50C460546F8F718
:10F00000F7FC012802D043F2020070BD21004FF04E
:10F010000000FAD028467EDF70BD00002DE9F74FD2
:10F020008AB0924688460A98F8F7E2FC06464FF600
:10F03000FF7900244D4627460A98FEF75BFB83467E
:10F04000202101A8F7F739FA012E01D0DEB105E041
:10F050002F48002201790A98F8F712FDB8F1000F45
:10F0600016D098F80000C00714D00A98FAF7E0FF0D
:10F070000546484516D1FEF725F9054648450ED008
:10F080004FF0010B0CE043F202000DB0BDE8F08F31
:10F09000852721E01F48CDF810A008901CE003242C
:10F0A0006CB121E0012E0AD10A98F7F767FD30B95B
:10F0B0000A98FFF7FBFB0A98F7F760FD50B101A82B
:10F0C00000905346324629460A98FFF72DFB04006C
:10F0D00002D009E0852712E0012E10D001AB0022FA
:10F0E00039460A987FDF044654EA07000DD0002213
:10F0F0005B4629460A98FFF789FB2046C5E701AB26
:10F10000424639460A987FDFEDE70122F0E700002A
:10F110000C2C0020443300203EB505460C466846C2
:10F12000FBF700FD6A4621462846FEF744F80948E9
:10F130000099C2682846FFF771FF04460146012284
:10F140002846FAF777F921462846009AF9F7F8FE9B
:10F150003EBD0000142C0020002805D103490120E9
:10F1600048700020F9F7D4BB7047000084330020BA
:10F1700010B51620F7F760FC48B10A4882684FF4D2
:10F18000800152B1016821F48001016010BDBDE829
:10F19000104042F20100F7F783BD4FF0E020C0F8C5
:10F1A000801110BD8035002010B51620F7F744FC03
:10F1B000A0B1114890F800044009082811D280B18C
:10F1C00001280ED004280CD00C4882684FF480012E
:10F1D0006AB1016841F48001016010BD42F2010092
:10F1E00001E042F20200BDE81040F7F759BD4FF0D0
:10F1F000E020C0F8001110BD16E000E080350020CE
:10F200002DE9F84F204D9246894606469846012240
:10F2100069461846AF68F9F76FFA58B300980021AD
:10F220000446801C09E000BF00EA07035AF82120C9
:10F2300005EB8303401C491CDA604145F4D34FEAD7
:10F24000164AF9F7B3FD4AEA0041601C384005EB65
:10F2500080003C4005EB8402C160D06866F3C500C5
:10F2600068F3891069F39F2020F00300401C20F010
:10F270000400D06095F8200402E000BFFCF7CCFC4D
:10F280000028FBD1BDE8F88F1838002070B50C00BD
:10F29000054602D10020F7F703FD15B90020F7F766
:10F2A000FFFC207828702088000A68702068000C15
:10F2B000A8702068000EE87020792871207A6871A3
:10F2C0002089000AA871A068000CE87170BD0000D8
:10F2D0002DE9F84F1D4C00256846D4E901A6F9F741
:10F2E0006FFD002738B30023009A61681CE0D1F855
:10F2F00000C00846944503D9ACEB02020A6015E051
:10F30000A2EB0C0263440760D0F80CC0C1698146CF
:10F31000BCF1000F08D006EB030828F07F48C0E9D5
:10F32000018CC9F81C5005460029E0D128466160CF
:10F33000FBF70EF903E02846FBF70AF910B1504637
:10F34000F9F708FBE770BDE8F88F0000B82C002043
:10F350000D4B10B5596831B102680C68A24204D84F
:10F36000A21A0A60C161586010BD0B4603E00B464B
:10F37000C969121B21B10C689442F8D3A41A0C601D
:10F380000260C161D86110BDB82C00202DE9F041A8
:10F39000144E77683D462C4603E0844204D025464F
:10F3A000E469002CF9D11BE0D4B1A5420BD1F86976
:10F3B000706040B90C49012088600021B160F07094
:10F3C0002F20FDF7C3F92168E069E86110B10268F8
:10F3D000114401607068874202D00120BDE8F081CD
:10F3E0000020FBE7B82C0020001001407CB5064649
:10F3F00000240D468DF800406846F7F7EDFC01A8A3
:10F4000000F0E6FA70B10570094946609DF8040005
:10F4100048709DF80000F7F703FD1420F7F7AAF9EC
:10F4200020467CBD04249DF80000F7F7F9FCF7E7BF
:10F43000743400202DE9F041194D6C68002C2CD05B
:10F44000184800270068A968B846401A20F07F468F
:10F450002068B0420CD82146361A0744E469087C7B
:10F4600020B181F81080886949698847002CEFD164
:10F4700029786878814206D1401CC0B268700228A1
:10F4800001D185F80180064869780C3040F8217078
:10F49000BDE8F0411420F7F76DB9BDE8F081000038
:10F4A000B82C00200415014010B5F7F717FC08B17F
:10F4B000F7F7F6FB134A01211348F7F7FDFB08B1F4
:10F4C000F7F7EEFB1048114A0121001DF7F7F4FB96
:10F4D00008B1F7F7E5FB0C480D4A01210830F7F7B2
:10F4E000EBFB08B1F7F7DCFB07480A4A01210C30B7
:10F4F000F7F7E2FB002803D0BDE81040F7F7D0BBD8
:10F5000010BD0000BD71020010FF0200B99B020097
:10F5100091E4020031E9020070B50C4605464FF453
:10F520008E71FDF7C8F8216AA068415C206A401C12
:10F530002062C5F81C1570BD1FB500228DF8002093
:10F540000291816801914261D0E9001268469047BA
:10F550001FBD00001FB50A4601788DF800104168F4
:10F560000191017A8DF80810C0680390044850F8A2
:10F570002210083850F82220684690471FBD00002E
:10F58000802C00200149012008707047342D002094
:10F5900010B588B0044620220E496846F6F766FF8B
:10F5A00006200090C01F0190029003904FF0EB7076
:10F5B00006900CB1084A00E0002269460748FBF7B4
:10F5C00079FD08B1F7F76CFB0448001F447008B0E0
:10F5D00010BD0000BC02030085F50200382D00209C
:10F5E0002DE9FF470C4605464FF40071FDF769F819
:10F5F00001274FF40178002618B34FF49279494659
:10F600002846FDF753F8E0B149462846FDF753F880
:10F61000C5F8088394F8290000B96F6002208DF8BE
:10F620000000D5F88004C5F880040390A06902901A
:10F63000E0680190A661E661D4E90012684690474F
:10F6400028E004212846FDF73CF818B34FF48471F4
:10F650002846FDF72BF8E8B121462846FEF77AFF49
:10F66000616AA069884215D1E06938B1E268616ACF
:10F67000A0612069E6616662E06008E094F8290014
:10F6800000B96F60C5F80883A661E268616A204628
:10F69000FEF779FF4FF48E7841462846FDF706F8CD
:10F6A00078B1206A6169884202D294F8280020B3B8
:10F6B00041462846FCF7FFFF616911B12046FFF77C
:10F6C0003BFF4FF4A27841462846FCF7EFFF0028A5
:10F6D00018D041462846FCF7EEFF94F8290000B107
:10F6E0002F60A06900280DD0A661E268616A04B0AD
:10F6F0002046BDE8F047FEF746BF21462846FFF703
:10F700000BFFDEE7BDE8FF871FB50A4601788DF8DD
:10F71000001041680191017A8DF80810C0680390CB
:10F72000044850F82210083850F8222068469047C4
:10F730001FBD0000802C00202DE9FF410C464FF436
:10F74000927705463946FCF7C2FF0026C0B139461C
:10F750002846FCF7C1FF02208DF80000D5F8800490
:10F76000C5F880040390D5F83C058DF80800E068E2
:10F770000190A661E661D4E900126846904723E053
:10F780004FF4887739462846FCF7A1FFE0B13946A7
:10F790002846FCF7A1FFD5F83C15A069884213D193
:10F7A000E06960B1E268D5F8000220F02000C5F8F9
:10F7B0000002E069A0612069E661E06001E0A66105
:10F7C000E2682046FEF7EAFE4FF4A2773946284663
:10F7D000FCF77DFF60B139462846FCF77DFFA06944
:10F7E00030B1A661D5F83C152046E268FEF7D6FE9A
:10F7F0004FF4907739462846FCF769FF002813D06C
:10F8000039462846FCF768FF606900280CD0D5F817
:10F810004C058DF800608DF80800A06801906661C5
:10F82000D4E9001268469047BDE8FF810870000ADD
:10F83000487002207047000010B514210448F6F704
:10F840003CFE04480068FBF78FF9002010BD000063
:10F85000F8360020200103002DE9F05F8346DDE942
:10F860000A4A994690460D460846012703E000BF24
:10F87000B0FBF8F07F1C4045FAD2B94500D94F469D
:10F880005FEACA7012D18CB15FEA8A7002D5B9F111
:10F89000000F01D0202607E0302605E0314658460B
:10F8A000641EF8F771FF0CB1A742F7D35FF00106B1
:10F8B000B9F1010F02D9A9F1010903E0B5FBF6F096
:10F8C000404502D306FB08F6F2E7DFF83C9000BFA4
:10F8D000B5FBF6F000FB165519F800105846F8F77E
:10F8E00053FFB6FBF8F6002EF2D15FEACA7009D0DA
:10F8F000002C07D0A74205D220215846641EF8F7F5
:10F9000043FFF5E7BDE8F09FB00003000348002285
:10F9100001498078F8F756B8158C0200D42B0020E6
:10F92000F8B5054680B2FAF72FFC040013D0154E47
:10F93000207A0027317B88420ED2A8B204F10A0156
:10F9400075DF28B1112806D0BDE8F840FEF7C0BF2A
:10F95000207A401C2072F8BD2772307C38B1A8B2E2
:10F960003B2176DF18B1082801D0FEF7B1FF71699D
:10F970000029F0D08DF80070ADF802506846884735
:10F98000F8BD000094300020417939B190F8B210F0
:10F9900021B990F8B40008B10120704700207047E9
:10F9A00001460148FBF767B9B030002030B4044687
:10F9B000007A00280AD06088002166DF28B111286B
:10F9C00002D0616830BC08470120207230BC70470B
:10F9D0000A494A788B78521CD2B2934200D1002255
:10F9E0000B78934201D1002070470270487800EBF9
:10F9F000400001EBC000001D70470000743400207F
:10FA00002DE9FC411646DDE90854CDE900541F46B6
:10FA10008046022200F00CF8002807D1CDE90054FE
:10FA20003B4610223146404600F002F8BDE8FC811A
:10FA30002DE9FC5F0026DDE90C4B994692468E4687
:10FA400080462788354630E0D8F80400002200EBD5
:10FA5000850069460068019001A864DF002830D164
:10FA60009DF8000050451FD10EB1002100E0022199
:10FA7000228808441118594522D846B9521C90B220
:10FA8000208009F800E02088401C20800126218881
:10FA900001A801EB0902694664DF002811D1208822
:10FAA0009DF80010084420806D1CB8F80000A842A2
:10FAB000CADC56B12088C01B401E80B2FF2802D984
:10FAC0000C20BDE8FC9F09F807000020F9E70000C2
:10FAD00010B504281DD209B1032400E00024F8F772
:10FAE00071FB202802D24FF0A04102E00A4900F049
:10FAF0001F0001EB8000D0F8001721F44031C0F85E
:10FB00000017D0F8001741EA0441C0F800170020A0
:10FB100010BD062010BD00000003005000207047FB
:10FB20002DE9F84F114D884681461E461746694615
:10FB3000DDF828A02868FBF732F8040013D01C2158
:10FB4000F6F7BBFC00202071C4F80090C4E90486DD
:10FB5000C4E902A769462868FBF742F8FEF744FBB0
:10FB60000020BDE8F88F0420FBE70000200103001F
:10FB700082780121012A0BD0062A09D0072A06D053
:10FB8000082A06D1416889880931890800E01421D2
:10FB9000018070471CB50446002000900190A078B9
:10FBA0008DF80200617B1A48FDF74AFF020017D06A
:10FBB000237BA1786846FDF7A3FD6846FFF7D8FFD1
:10FBC000208804F1080369466268FDF717FD48B113
:10FBD000072806D001210F4A112808D086280FD007
:10FBE00003201CBDA17B21F00301A1731CBDA07BE0
:10FBF00020F0010040F00200A073117000201CBD35
:10FC0000A37B23F0020343F00103A37311701CBD17
:10FC1000C8320020F82B002038B505460C460020DD
:10FC200001E00098401C00906946284600F00EF85C
:10FC300000280AD08178A142F3D1817B8A07F0D4D1
:10FC4000C907EED181680029EBD138BD10B5084B4A
:10FC50000A6809E003EB02142488844203D103EB11
:10FC600002100A6010BD521C022AF3D3002010BDFE
:10FC7000D83200204FF6FF710180FF21817041735F
:10FC8000817B21F003018173002101734160816058
:10FC90007047000070B50546002406E0687B2044EC
:10FCA000C1B20648FDF7E0FE641C287BA042F5D8EF
:10FCB0002846BDE87040FFF7DDBF0000C8320020D5
:10FCC0002DE9FC47064636489846144600780D460E
:10FCD0004FF0000978B37DB32888A0F57F41FF3944
:10FCE00031D0688848B36868FAF746FB68B374B3E4
:10FCF0002088ADF80000678801A8FEF7A7F9040086
:10FD00002FD084F800804FF0000A84F816A0BDF8C8
:10FD10000000A08268682061214801210C38FAF7B0
:10FD2000C8FFE060288820816888A080E780B8F15B
:10FD3000030F1DD020E001E003E004E00220BDE855
:10FD4000FC870520FBE70420F9E70320F7E7FFE73E
:10FD50002889694687B2384600F0ACF80028EED111
:10FD6000CAE7BDF80010384600F098F80820E6E72A
:10FD70000420A0753068A061A4F80A9001A8FEF7DD
:10FD800073F946B1C6F804A0E1680648316086F808
:10FD90000AA000893081FEF719FA0020CFE70000A1
:10FDA000002D00205C3600202DE9F8430D46898A9D
:10FDB000374A01EB810102EB810630B1294630461A
:10FDC000FDF7FEF80120BDE8F88331897068002452
:10FDD00000EB81072E48A97DA8384FF00E080729AF
:10FDE0004ED2DFE801F00D2D162404404A00446095
:10FDF000A969016026482749A838FEF7A5FA30B15D
:10FE00000220A875042339462A1D009423E00A2005
:10FE1000D9E728692A4608B1032000E0012090753F
:10FE2000042305F10C0207F10801009413E00120FE
:10FE3000A8750094E88807F10C0183002A690AE09C
:10FE400028782A4603280CD006209075042305F153
:10FE50000802391D00941048FBF7D6FBA8B14446B0
:10FE60000FE00520F1E70621A9750A4940680988D5
:10FE7000FEF7E8FA040004D107E041F61D5400E063
:10FE80000F2429463046FDF79BF820469BE70000EB
:10FE900034360020E02C0020B02D002001EB810240
:10FEA000034901EB82014A89101AC01E488170473C
:10FEB0003436002070B5C01C82B240F2FE3082425F
:10FEC00001D3092070BD114B00204FF4806500BFA5
:10FED00000EB800413F8246096B903EB84063489A0
:10FEE000768914443444A4B2AC4209D2088000EBB1
:10FEF000800003EB8000418911444181002070BDE6
:10FF0000401C80B20228E3D3072070BD34360020A5
:10FF1000082E0020282E0020482E0020682E0020C9
:10FF20000D0E0F100B0C1819F42F002014300020A8
:10FF3000403000200B000300618302000C0003002E
:10FF400061830200180003006183020019000300AE
:10FF500061830200070000000000000000000000B4
:10FF6000000000000000000006000000000000008B
:10FF70000000000000000000000000001000000071
:10FF80000000000000000000000000000000000071
:10FF90001100000000000000000000000000000050
:10FFA000000000000100000001000100A4FF0200A9
:10FFB00001000100B8FF02000000000095DB020014
:10FFC00011980200770A000000000000770A000084
:10FFD000000000007ADA00000000000051D20200A8
:10FFE000070000000000000000000000000000000A
:10FFF0000000000095DC0200B1ED0200119B020040
:020000040003F7
:1000000091980200010000000000000001000600BD
:10001000082C00203DEE020001000000000000005E
:1000200000000000000000000000000007000000C9
:1000300000000000000000000000000000000000C0
:1000400003000000000000000000000000000000AD
:10005000000000000500000000000000000000009B
:10006000000000000000000021DF0200000000503E
:1000700000030050BDC9020019CC020003000000BB
:1000800054340020000000000000000000000000C8
:100090000338FDD870470000CC2C00200000FFFF83
:1000A000DEC0ADDEFF011EF1DEC0ADDEFE011EF1E1
:1000B000303132333435363738394142434445469E
:1000C0006E72665F6673746F726167655F696E6991
:1000D00074006E72665F6673746F726167655F75D8
:1000E0006E696E6974006E72665F6673746F7261BA
:1000F00067655F72656164006E72665F6673746FD8
:10010000726167655F7772697465006E72665F66BB
:1001100073746F726167655F65726173650000007B
:10012000102D00200010000004000000010000005D
:100130008DA0020039F8020035E2020021FB020026
:100140000D8E02008DE402001DFB020011A30200CF
:10015000000000000000000000000000000000009F
:1001600000000000000000005001030068010300CF
:1001700004000000556E6B6E6F776E206572726FB3
:100180007220636F646500000000000074080300C3
:100190000100000020070300020000001405030016
:1001A000030000009407030004000000E8070300B8
:1001B00005000000C80603000600000064060300F6
:1001C00007000000D007030008000000DC06030061
:1001D00009000000400703000A0000005C0803005B
:1001E0000B000000FC0403000C000000F4060300F8
:1001F0000D000000C40803000E000000C00703004B
:100200000F000000FC07030010000000300803008E
:1002100011000000D808030012000000AC08030021
:100220001300000048080300800000007C06030063
:1002300081000000B805030082000000780503007B
:1002400083000000580503008400000094050300AB
:1002500085000000A006030086000000A807030038
:1002600090000000440603009100000038050300E0
:10027000920000000807030000820000100803003D
:10028000018200005C07030002820000780703007F
:1002900000840000D40503000184000080080300EE
:1002A000028400001C06030003840000F80503001C
:1002B000B5BB020089BB020081BB0200FFFFFFFF4C
:1002C000FFFFFFFFFFFFFFFFFFFFFFFF000000003A
:1002D000000000000000D60107010000E80C030048
:1002E000F00C030000000000000000000100000707
:1002F000DC020300EC02030008000000140303000A
:100300002403030008000000240303003403030057
:1003100008000000180D0300280D03000000000075
:1003200000000000080D0300180D0300000000008D
:1003300000000000980C0300A00C0300A00C0300B8
:10034000C80C0300C80C0300E00C0300E00C030021
:10035000E80C0300882B002034030300540303003F
:1003600008000000F00C0300000D0300000D030066
:10037000080D030064030300740303000800000079
:1003800000404040404040404040414141414140A8
:10039000404040404040404040404040404040405D
:1003A00040050202020202020202020202020202EC
:1003B00002202020202020202020200202020202F1
:1003C0000202909090909090101010101010101049
:1003D0001010101010101010101010100202020255
:1003E0000202888888888888080808080808080899
:1003F0000808080808080808080808080202020295
:10040000400000008103030073645F626C655F67F6
:1004100061705F646174615F6C656E6774685F755D
:10042000706461746528292028726571756573741C
:1004300029206F6E20636F6E6E656374696F6E2026
:10044000307825782072657475726E656420257326
:100450002E000000546865207265717565737465BF
:100460006420636F6D62696E6174696F6E206F6680
:1004700020545820616E64205258207061636B656F
:1004800074206C656E6774687320697320746F6F75
:10049000206C6F6E67206279202575206D6963720C
:1004A0006F7365636F6E64732E0000006164647225
:1004B0005F69735F77697468696E5F626F756E6498
:1004C0007328705F66732C20706167655F61646478
:1004D000722C20286C656E202A20705F66732D3E7A
:1004E000705F666C6173685F696E666F2D3E6572E2
:1004F0006173655F756E6974292900004E52465F0D
:100500004552524F525F494E56414C49445F444117
:10051000544100004E52465F4552524F525F534F76
:1005200046544445564943455F4E4F545F454E41FE
:10053000424C4544000000004E52465F4552524F27
:10054000525F464541545552455F4E4F545F454EAC
:1005500041424C45440000004E52465F4552524FC6
:10056000525F4D555445585F554E4C4F434B5F4677
:1005700041494C45440000004E52465F4552524F9F
:10058000525F4D555445585F4C4F434B5F46414970
:100590004C4544004E52465F4552524F525F4D55B6
:1005A0005445585F434F4E445F494E49545F46415E
:1005B000494C4544000000004E52465F4552524FA0
:1005C000525F4D555445585F494E49545F46414925
:1005D0004C4544004E52465F4552524F525F424C8A
:1005E000455F495053505F52585F504B545F5452CF
:1005F000554E4341544544004E52465F4552524F7A
:10060000525F424C455F495053505F504545525FE1
:1006100052454A4543544544000000004E52465F4F
:100620004552524F525F424C455F495053505F4CC8
:10063000494E4B5F444953434F4E4E454354454406
:10064000000000004E52465F4552524F525F4150EB
:10065000495F4E4F545F494D504C454D454E5445B2
:10066000440000004E52465F4552524F525F4E4F7B
:10067000545F535550504F52544544004E52465FBC
:100680004552524F525F4D4F44554C455F4E4F546B
:100690005F494E495449414C495A454400000000C5
:1006A0004E52465F4552524F525F4D4F44554C4556
:1006B0005F414C52454144595F494E495449414C70
:1006C000495A4544000000004E52465F4552524F81
:1006D000525F4E4F545F464F554E44004E52465F58
:1006E0004552524F525F494E56414C49445F535414
:1006F000415445004E52465F4552524F525F44416D
:1007000054415F53495A45004E52465F4552524F3D
:10071000525F494F5F50454E44494E47000000002C
:100720004E52465F4552524F525F5356435F4841C7
:100730004E444C45525F4D495353494E47000000CB
:100740004E52465F4552524F525F494E56414C49B8
:10075000445F4C454E475448000000004E52465FEF
:100760004552524F525F4452565F5457495F45526B
:10077000525F414E41434B004E52465F4552524FED
:10078000525F4452565F5457495F4552525F444E40
:1007900041434B004E52465F4552524F525F494EC5
:1007A0005445524E414C00004E52465F4552524F06
:1007B000525F53544F524147455F46554C4C0000E1
:1007C0004E52465F4552524F525F4E554C4C0000C0
:1007D0004E52465F4552524F525F494E56414C4928
:1007E000445F504152414D004E52465F4552524F78
:1007F000525F4E4F5F4D454D000000004E52465F28
:100800004552524F525F464F5242494444454E0072
:100810004E52465F4552524F525F4452565F5457B4
:10082000495F4552525F4F56455252554E000000A7
:100830004E52465F4552524F525F494E56414C49C7
:10084000445F4144445200004E52465F4552524F6D
:10085000525F5245534F5552434553004E52465FE7
:100860004552524F525F494E56414C49445F464CA7
:10087000414753004E52465F53554343455353003F
:100880004E52465F4552524F525F424C455F49506F
:1008900053505F4348414E4E454C5F414C52454199
:1008A00044595F4558495354530000004E52465F27
:1008B0004552524F525F434F4E4E5F434F554E5439
:1008C000000000004E52465F4552524F525F54495D
:1008D0004D454F55540000004E52465F4552524F11
:1008E000525F4255535900007761726E696E67001E
:1008F00064656275670000001B5B313B33306D003F
:100900001B5B306D000000001B5B313B33316D0021
:100910001B5B313B33326D001B5B313B33336D006E
:100920001B5B313B33346D001B5B313B33356D005A
:100930001B5B313B33366D001B5B313B33376D0046
:10094000696E666F000000006572726F72000000D1
:1009500073645F626C655F6366675F7365742829A3
:100960002072657475726E656420257320776865E2
:100970006E20617474656D7074696E6720746F2089
:1009800073657420424C455F47415454535F43465E
:10099000475F534552564943455F4348414E47459B
:1009A000442E000073645F626C655F6366675F730B
:1009B000657428292072657475726E6564202573CC
:1009C000207768656E20617474656D7074696E67F8
:1009D00020746F2073657420424C455F434F4D4D2A
:1009E0004F4E5F4346475F56535F555549442E006F
:1009F00073645F626C655F6366675F736574282903
:100A00002072657475726E65642025732077686541
:100A10006E20617474656D7074696E6720746F20E8
:100A200073657420424C455F47415454535F4346BD
:100A3000475F415454525F5441425F53495A452ED7
:100A40000000000073645F626C655F6366675F73DC
:100A5000657428292072657475726E65642025732B
:100A6000207768656E20617474656D7074696E6757
:100A700020746F2073657420424C455F434F4E4E87
:100A80005F4346475F4741502E00000073645F623A
:100A90006C655F6366675F7365742829207265748F
:100AA00075726E6564202573207768656E206174A9
:100AB00074656D7074696E6720746F20736574203F
:100AC000424C455F4741505F4346475F524F4C455C
:100AD0005F434F554E542E0073645F626C655F63D5
:100AE00066675F73657428292072657475726E6518
:100AF00064202573207768656E20617474656D705D
:100B000074696E6720746F2073657420424C455F72
:100B1000434F4E4E5F4346475F474154542E0000BB
:100B20006E72665F626C655F6761747400000000DE
:100B3000626C655F62617300636C6F636B000000E1
:100B4000434C4F434B0000004750494F5445000071
:100B50005052530055415254000000005541525428
:100B60004500000061746669666F2E6D5F71756582
:100B7000756500006E72665F6673746F726167659B
:100B80000000000061746669666F2E6D5F666966BD
:100B90006F0000007077725F6D676D740000000079
:100BA00062616C6C6F632E6C6F675F6D656D706FEB
:100BB0006F6C0000617070006E72665F7364680035
:100BC0006E72665F7364685F626C65006E72665F0A
:100BD0007364685F736F6300280D0300882B002027
:100BE000800200003C650200900D0300082E0020EA
:100BF000382E0000286A0200200B030000000303C7
:100C0000300B030000000000380B03000000000060
:100C1000400B030000000000480B03000000000030
:100C2000500B030000000000540B03000000000004
:100C30005C0B030000000000640B030000000003D5
:100C4000740B030000000303840B03000000000387
:100C5000940B030000000000A00B03000000000341
:100C6000B40B030000000303B80B030000000303F0
:100C7000C00B030000000303CC0B030000000303C0
:100C8000602D0020582D0020602D002058370020B6
:100C9000F42D002018000000897E020000000000F2
:100CA000F5AD0200EC2E0020D57402000C2F0020C0
:100CB0001D7D0200000000008D7D0200000000008C
:100CC0008D7F0200000000006F800200882E00204F
:100CD000DF780200D82E002077AF0200002F00201E
:100CE000617C0200000000002DB502000000000041
:100CF00059F102000000000065B50200000000008C
:100D00003F7502000C2F002061C4020000000000AB
:100D1000D5C5020000000000D9E502000000000077
:100D200045B50200000000001201031CFFFF140D76
:100D300018011A0F041A0A040128042D91DB022A53
:100D400018017909390A01BD13E42D0240200A1A5D
:100D5000EC441220AA40080425B0020314480903F9
:100D600014E808031A40081AF0081119081AF808BC
:100D70001A08081A10041A18041A20041A28041A47
:100D800030041A3804517B90D061044DB9940200AC
:040000050002620192
:00000001FF
